******************************************************************************
               TMS320C6x Linker PC v8.1.4                      
******************************************************************************
>> Linked Thu Sep 21 16:29:36 2017

OUTPUT FILE NAME:   <Test_bios.out>
ENTRY POINT SYMBOL: "_c_int00"  address: 80009760


MEMORY CONFIGURATION

         name            origin    length      used     unused   attr    fill
----------------------  --------  ---------  --------  --------  ----  --------
  L2SRAM                00800000   00040000  00000000  00040000  RW X
  OCMC_RAM1             40300000   00080000  00000000  00080000  RW X
  OCMC_RAM2             40400000   00100000  00000000  00100000  RW X
  OCMC_RAM3             40500000   00100000  00000000  00100000  RW X
  EXT_RAM               80000000   80000000  00013f8e  7ffec072  RWIX


SEGMENT ALLOCATION MAP

run origin  load origin   length   init length attrs members
----------  ----------- ---------- ----------- ----- -------
80000000    80000000    0000f5ca   0000f5ca    r-x
  80000000    80000000    0000c840   0000c840    r-x .text
  8000c840    8000c840    00002d8a   00002d8a    r-- .const
8000f5d0    8000f5d0    00004368   00000000    rw-
  8000f5d0    8000f5d0    00002000   00000000    rw- .stack
  800115d0    800115d0    00001c08   00000000    rw- .far
  800131d8    800131d8    0000063c   00000000    rw- .fardata
  80013818    80013818    00000120   00000000    rw- .cio
80013c00    80013c00    00000660   00000660    r-x
  80013c00    80013c00    00000200   00000200    r-x .vecs
  80013e00    80013e00    00000460   00000460    r-- .cinit


SECTION ALLOCATION MAP

 output                                  attributes/
section   page    origin      length       input sections
--------  ----  ----------  ----------   ----------------
.stack     0    8000f5d0    00002000     UNINITIALIZED
                  8000f5d0    00000008     boot.ae66 : boot.oe66 (.stack)
                  8000f5d8    00001ff8     --HOLE--

.cinit     0    80013e00    00000460     
                  80013e00    0000043c     (.cinit..fardata.load) [load image, compression = rle]
                  8001423c    0000000c     (__TI_handler_table)
                  80014248    00000008     (.cinit..far.load) [load image, compression = zero_init]
                  80014250    00000010     (__TI_cinit_table)

.init_array 
*          0    80000000    00000000     UNINITIALIZED

.text      0    80000000    0000c840     
                  80000000    00000880     ti.targets.rts6000.ae66 : System.oe66 (.text:xdc_runtime_System_doPrint__I)
                  80000880    000007e0     sysbios.ae66 : BIOS.obj (.text:ti_sysbios_knl_Semaphore_pend__E)
                  80001060    00000780                  : BIOS.obj (.text:ti_sysbios_family_c64p_Exception_handler__I)
                  800017e0    00000640                  : BIOS.obj (.text:ti_sysbios_heaps_HeapMem_allocUnprotected__E)
                  80001e20    000005c0                  : BIOS.obj (.text:ti_sysbios_heaps_HeapMem_freeUnprotected__E)
                  800023e0    000004c0                  : BIOS.obj (.text:ti_sysbios_knl_Task_Instance_finalize__E)
                  800028a0    00000480                  : BIOS.obj (.text:ti_sysbios_knl_Task_sleep__E)
                  80002d20    000003c0                  : BIOS.obj (.text:ti_sysbios_timers_dmtimer_Timer_checkFreq__I)
                  800030e0    000003a0                  : BIOS.obj (.text:ti_sysbios_knl_Task_Instance_init__E)
                  80003480    00000380                  : BIOS.obj (.text:ti_sysbios_timers_dmtimer_Timer_deviceConfig__I)
                  80003800    00000300                  : BIOS.obj (.text:ti_sysbios_knl_Task_Module_startup__E)
                  80003b00    000002e0                  : BIOS.obj (.text:ti_sysbios_heaps_HeapMem_Instance_init__E)
                  80003de0    000002a0                  : BIOS.obj (.text:ti_sysbios_knl_Clock_workFunc__E)
                  80004080    000002a0                  : BIOS.obj (.text:ti_sysbios_knl_Semaphore_post__E)
                  80004320    00000280                  : BIOS.obj (.text:ti_sysbios_timers_dmtimer_Timer_setPeriodMicroSecs__E)
                  800045a0    00000280     ti.targets.rts6000.ae66 : LoggerBuf.oe66 (.text:xdc_runtime_LoggerBuf_write8__E)
                  80004820    00000260     sysbios.ae66 : BIOS.obj (.text:ti_sysbios_family_c64p_Hwi_dispatchCore__I)
                  80004a80    00000240     rts6600_elf.lib : imath64.obj (.text:__c6xabi_divull)
                  80004cc0    00000240     sysbios.ae66 : BIOS.obj (.text:ti_sysbios_family_c64p_Exception_internalHandler__I)
                  80004f00    00000240     app_pe66.oe66 (.text:xdc_runtime_System_printfExtend__I)
                  80005140    00000220     sysbios.ae66 : BIOS.obj (.text:ti_sysbios_knl_Swi_run__I)
                  80005360    00000220     ti.targets.rts6000.ae66 : Core-mem.oe66 (.text:xdc_runtime_Core_createObject__I)
                  80005580    00000200     sysbios.ae66 : c64p_Hwi_disp_always.obj (.text:_ti_sysbios_family_c64p_Hwi_dispatchAlways)
                  80005780    000001e0                  : BIOS.obj (.text:ti_sysbios_gates_GateMutex_enter__E)
                  80005960    000001e0                  : BIOS.obj (.text:ti_sysbios_knl_Task_checkStacks__E)
                  80005b40    000001e0                  : BIOS.obj (.text:ti_sysbios_knl_Task_exit__E)
                  80005d20    000001e0     ti.targets.rts6000.ae66 : Error.oe66 (.text:xdc_runtime_Error_policyDefault__E)
                  80005f00    000001e0                             : Startup.oe66 (.text:xdc_runtime_Startup_startMods__I)
                  800060e0    000001c0                             : LoggerBuf.oe66 (.text:xdc_runtime_LoggerBuf_write4__E)
                  800062a0    000001c0                             : Text.oe66 (.text:xdc_runtime_Text_putSite__E)
                  80006460    000001a0     sysbios.ae66 : BIOS.obj (.text:ti_sysbios_family_c66_Cache_getL2InitSize__I)
                  80006600    000001a0                  : BIOS.obj (.text:ti_sysbios_knl_Task_schedule__I)
                  800067a0    00000180                  : c64p_Exception_asm.obj (.text)
                  80006920    00000180                  : BIOS.obj (.text:ti_sysbios_family_c66_Cache_block__I)
                  80006aa0    00000180                  : BIOS.obj (.text:ti_sysbios_knl_Task_startCore__E)
                  80006c20    00000180                  : BIOS.obj (.text:ti_sysbios_timers_dmtimer_Timer_start__E)
                  80006da0    00000180     ti.targets.rts6000.ae66 : Core-smem.oe66 (.text:xdc_runtime_Core_constructObject__I)
                  80006f20    00000160     sysbios.ae66 : BIOS.obj (.text:ti_sysbios_knl_Swi_post__E)
                  80007080    00000160                  : BIOS.obj (.text:ti_sysbios_knl_Task_postInit__I)
                  800071e0    00000140     boot.ae66 : autoinit.oe66 (.text:_auto_init_elf)
                  80007320    00000140     sysbios.ae66 : BIOS.obj (.text:ti_sysbios_family_c64p_Hwi_Module_startup__E)
                  80007460    00000140                  : BIOS.obj (.text:ti_sysbios_family_c66_Cache_getL1DInitSize__I)
                  800075a0    00000140                  : BIOS.obj (.text:ti_sysbios_family_c66_Cache_getL1PInitSize__I)
                  800076e0    00000140                  : BIOS.obj (.text:ti_sysbios_family_c66_Cache_startup__I)
                  80007820    00000140                  : BIOS.obj (.text:ti_sysbios_knl_Semaphore_Instance_init__E)
                  80007960    00000140                  : BIOS.obj (.text:ti_sysbios_knl_Task_blockI__E)
                  80007aa0    00000120                  : BIOS.obj (.text:ti_sysbios_knl_Swi_restoreHwi__E)
                  80007bc0    00000120                  : BIOS.obj (.text:ti_sysbios_timers_dmtimer_Timer_Module_startup__E)
                  80007ce0    00000120                  : BIOS.obj (.text:ti_sysbios_timers_dmtimer_Timer_initDevice__I)
                  80007e00    00000120     ti.targets.rts6000.ae66 : Core-mem.oe66 (.text:xdc_runtime_Core_deleteObject__I)
                  80007f20    00000120                             : LoggerBuf.oe66 (.text:xdc_runtime_LoggerBuf_setFilterLevel__E)
                  80008040    00000120                             : Text.oe66 (.text:xdc_runtime_Text_putLab__E)
                  80008160    00000120                             : Text.oe66 (.text:xdc_runtime_Text_putMod__E)
                  80008280    00000100     rts6600_elf.lib : copy_decompress_rle.obj (.text:__TI_decompress_rle_core)
                  80008380    00000100     sysbios.ae66 : BIOS.obj (.text:ti_sysbios_knl_Swi_schedule__I)
                  80008480    00000100                  : BIOS.obj (.text:ti_sysbios_knl_Task_unblockI__E)
                  80008580    00000100     ti.targets.rts6000.ae66 : LoggerBuf.oe66 (.text:xdc_runtime_LoggerBuf_getFilterLevel__E)
                  80008680    00000100                             : Startup.oe66 (.text:xdc_runtime_Startup_exec__E)
                  80008780    000000e0     rts6600_elf.lib : trgdrv.obj (.text:HOSTwrite)
                  80008860    000000e0                     : memset.obj (.text:memset)
                  80008940    000000e0     sysbios.ae66 : BIOS.obj (.text:ti_sysbios_knl_Swi_runLoop__I)
                  80008a20    000000e0                  : BIOS.obj (.text:ti_sysbios_knl_Swi_startup__E)
                  80008b00    000000e0                  : BIOS.obj (.text:ti_sysbios_timers_dmtimer_Timer_startup__E)
                  80008be0    000000e0     ti.targets.rts6000.ae66 : Error.oe66 (.text:xdc_runtime_Error_print__E)
                  80008cc0    000000e0                             : Memory.oe66 (.text:xdc_runtime_Memory_alloc__E)
                  80008da0    000000e0                             : Text.oe66 (.text:xdc_runtime_Text_visitRope2__I)
                  80008e80    000000c0     rts6600_elf.lib : divu.obj (.text:__divu)
                  80008f40    000000c0                     : exit.obj (.text:exit)
                  80009000    000000c0     main.obj (.text)
                  800090c0    000000c0     sysbios.ae66 : BIOS.obj (.text:ti_sysbios_heaps_HeapMem_alloc__E)
                  80009180    000000c0                  : BIOS.obj (.text:ti_sysbios_heaps_HeapMem_getStats__E)
                  80009240    000000c0                  : BIOS.obj (.text:ti_sysbios_knl_Clock_logTick__E)
                  80009300    000000c0                  : BIOS.obj (.text:ti_sysbios_knl_Task_allBlockedFunction__I)
                  800093c0    000000c0     app_pe66.oe66 (.text:ti_sysbios_knl_Task_create)
                  80009480    000000c0     sysbios.ae66 : BIOS.obj (.text:ti_sysbios_timers_dmtimer_Timer_stop__E)
                  80009540    000000c0     rts6600_elf.lib : tls.obj (.text:tls:init:__TI_tls_init)
                  80009600    000000c0     ti.targets.rts6000.ae66 : System.oe66 (.text:xdc_runtime_System_formatNum__I)
                  800096c0    000000a0     rts6600_elf.lib : remu.obj (.text:__remu)
                  80009760    000000a0     boot.ae66 : boot.oe66 (.text:_c_int00)
                  80009800    000000a0     rts6600_elf.lib : memcpy64.obj (.text:memcpy)
                  800098a0    000000a0     sysbios.ae66 : BIOS.obj (.text:ti_sysbios_family_c64p_Exception_Module_startup__E)
                  80009940    000000a0                  : BIOS.obj (.text:ti_sysbios_family_c64p_Hwi_dispatchC__I)
                  800099e0    000000a0                  : BIOS.obj (.text:ti_sysbios_family_c64p_Hwi_getStackInfo__E)
                  80009a80    000000a0                  : BIOS.obj (.text:ti_sysbios_heaps_HeapMem_init__I)
                  80009b20    000000a0     ti.targets.rts6000.ae66 : Assert.oe66 (.text:xdc_runtime_Assert_raise__I)
                  80009bc0    000000a0                             : Error.oe66 (.text:xdc_runtime_Error_setX__E)
                  80009c60    000000a0     app_pe66.oe66 (.text:xdc_runtime_LoggerBuf_Object__create__S)
                  80009d00    000000a0     ti.targets.rts6000.ae66 : SysMin.oe66 (.text:xdc_runtime_SysMin_abort__E)
                  80009da0    000000a0                             : SysMin.oe66 (.text:xdc_runtime_SysMin_flush__E)
                  80009e40    000000a0                             : SysMin.oe66 (.text:xdc_runtime_SysMin_putch__E)
                  80009ee0    000000a0                             : Text.oe66 (.text:xdc_runtime_Text_xprintf__I)
                  80009f80    00000080     rts6600_elf.lib : trgmsg.obj (.text:__TI_readmsg)
                  8000a000    00000080                     : trgmsg.obj (.text:__TI_writemsg)
                  8000a080    00000080                     : llshift.obj (.text:__c6xabi_llshl)
                  8000a100    00000080     sysbios.ae66 : c62_TaskSupport_asm.obj (.text:_ti_sysbios_family_c62_TaskSupport_swap__E)
                  8000a180    00000080     app_pe66.oe66 (.text:ti_sysbios_BIOS_atExitFunc__I)
                  8000a200    00000080     app_pe66.oe66 (.text:ti_sysbios_BIOS_registerRTSLock__I)
                  8000a280    00000080     app_pe66.oe66 (.text:ti_sysbios_gates_GateHwi_Object__create__S)
                  8000a300    00000080     app_pe66.oe66 (.text:ti_sysbios_gates_GateMutex_Object__create__S)
                  8000a380    00000080     sysbios.ae66 : BIOS.obj (.text:ti_sysbios_hal_Hwi_checkStack)
                  8000a400    00000080                  : BIOS.obj (.text:ti_sysbios_hal_Hwi_initStack)
                  8000a480    00000080     app_pe66.oe66 (.text:ti_sysbios_heaps_HeapMem_Object__create__S)
                  8000a500    00000080     app_pe66.oe66 (.text:ti_sysbios_knl_Clock_doTick__I)
                  8000a580    00000080     sysbios.ae66 : BIOS.obj (.text:ti_sysbios_knl_Idle_run__E)
                  8000a600    00000080                  : BIOS.obj (.text:ti_sysbios_knl_Semaphore_pendTimeout__I)
                  8000a680    00000080                  : BIOS.obj (.text:ti_sysbios_knl_Task_processVitalTaskFlag__I)
                  8000a700    00000080                  : BIOS.obj (.text:ti_sysbios_knl_Task_restore__E)
                  8000a780    00000080     ti.targets.rts6000.ae66 : Core-label.oe66 (.text:xdc_runtime_Core_assignLabel__I)
                  8000a800    00000080                             : Core-params.oe66 (.text:xdc_runtime_Core_assignParams__I)
                  8000a880    00000080                             : LoggerBuf.oe66 (.text:xdc_runtime_LoggerBuf_Instance_init__E)
                  8000a900    00000080                             : LoggerBuf.oe66 (.text:xdc_runtime_LoggerBuf_Module_startup__E)
                  8000a980    00000080                             : LoggerBuf.oe66 (.text:xdc_runtime_LoggerBuf_filterOutEvent__I)
                  8000aa00    00000080     app_pe66.oe66 (.text:xdc_runtime_SysMin_output__I)
                  8000aa80    00000080     ti.targets.rts6000.ae66 : System.oe66 (.text:xdc_runtime_System_atexit__E)
                  8000ab00    00000080                             : System.oe66 (.text:xdc_runtime_System_processAtExit__E)
                  8000ab80    00000080                             : System.oe66 (.text:xdc_runtime_System_putchar__I)
                  8000ac00    00000080                             : Text.oe66 (.text:xdc_runtime_Text_printVisFxn__I)
                  8000ac80    00000060     rts6600_elf.lib : llshift.obj (.text:__c6xabi_llshru)
                  8000ace0    00000060     sysbios.ae66 : c64p_Hwi_asm_switch.obj (.text:_ti_sysbios_family_c64p_Hwi_switchAndDispatch__I)
                  8000ad40    00000060                  : c64p_Hwi_asm_switch.obj (.text:_ti_sysbios_family_xxx_Hwi_switchAndRunFunc)
                  8000ada0    00000060     app_pe66.oe66 (.text:ti_sysbios_BIOS_errorRaiseHook__I)
                  8000ae00    00000060     app_pe66.oe66 (.text:ti_sysbios_BIOS_removeRTSLock__I)
                  8000ae60    00000060     app_pe66.oe66 (.text:ti_sysbios_BIOS_startFunc__I)
                  8000aec0    00000060     sysbios.ae66 : BIOS.obj (.text:ti_sysbios_family_c62_TaskSupport_start__E)
                  8000af20    00000060                  : BIOS.obj (.text:ti_sysbios_family_c66_Cache_Module_startup__E)
                  8000af80    00000060     app_pe66.oe66 (.text:ti_sysbios_gates_GateMutex_Object__delete__S)
                  8000afe0    00000060     sysbios.ae66 : BIOS.obj (.text:ti_sysbios_heaps_HeapMem_free__E)
                  8000b040    00000060                  : BIOS.obj (.text:ti_sysbios_knl_Clock_Module_startup__E)
                  8000b0a0    00000060     app_pe66.oe66 (.text:ti_sysbios_knl_Queue_construct)
                  8000b100    00000060     app_pe66.oe66 (.text:ti_sysbios_knl_Semaphore_construct)
                  8000b160    00000060     sysbios.ae66 : BIOS.obj (.text:ti_sysbios_knl_Swi_Module_startup__E)
                  8000b1c0    00000060                  : BIOS.obj (.text:ti_sysbios_knl_Task_enter__I)
                  8000b220    00000060     app_pe66.oe66 (.text:xdc_runtime_LoggerBuf_Object__delete__S)
                  8000b280    00000060     ti.targets.rts6000.ae66 : Memory.oe66 (.text:xdc_runtime_Memory_valloc__E)
                  8000b2e0    00000060                             : SysMin.oe66 (.text:xdc_runtime_SysMin_Module_startup__E)
                  8000b340    00000060                             : SysMin.oe66 (.text:xdc_runtime_SysMin_exit__E)
                  8000b3a0    00000060                             : System.oe66 (.text:xdc_runtime_System_avprintf__E)
                  8000b400    00000060                             : System.oe66 (.text:xdc_runtime_System_vprintf__E)
                  8000b460    00000060                             : Text.oe66 (.text:xdc_runtime_Text_cordText__E)
                  8000b4c0    00000040     rts6600_elf.lib : strasg.obj (.text:__strasgi_64plus)
                  8000b500    00000040                     : args_main.obj (.text:_args_main)
                  8000b540    00000040                     : imath64.obj (.text:_subcull)
                  8000b580    00000040     sysbios.ae66 : c62_TaskSupport_asm.obj (.text:_ti_sysbios_family_c62_TaskSupport_buildTaskStack)
                  8000b5c0    00000040     app_pe66.oe66 (.text:ti_sysbios_BIOS_exitFunc__I)
                  8000b600    00000040     app_pe66.oe66 (.text:ti_sysbios_BIOS_rtsLock__I)
                  8000b640    00000040     app_pe66.oe66 (.text:ti_sysbios_BIOS_rtsUnlock__I)
                  8000b680    00000040     sysbios.ae66 : BIOS.obj (.text:ti_sysbios_family_c64p_Hwi_disableInterrupt__E)
                  8000b6c0    00000040                  : BIOS.obj (.text:ti_sysbios_family_c64p_Hwi_enableInterrupt__E)
                  8000b700    00000040     app_pe66.oe66 (.text:ti_sysbios_gates_GateHwi_Handle__label__S)
                  8000b740    00000040     app_pe66.oe66 (.text:ti_sysbios_gates_GateHwi_Object__delete__S)
                  8000b780    00000040     app_pe66.oe66 (.text:ti_sysbios_gates_GateMutex_Handle__label__S)
                  8000b7c0    00000040     sysbios.ae66 : BIOS.obj (.text:ti_sysbios_gates_GateMutex_Instance_init__E)
                  8000b800    00000040                  : BIOS.obj (.text:ti_sysbios_gates_GateMutex_leave__E)
                  8000b840    00000040     app_pe66.oe66 (.text:ti_sysbios_heaps_HeapMem_Handle__label__S)
                  8000b880    00000040     app_pe66.oe66 (.text:ti_sysbios_heaps_HeapMem_Object__delete__S)
                  8000b8c0    00000040     app_pe66.oe66 (.text:ti_sysbios_heaps_HeapMem_Object__get__S)
                  8000b900    00000040     app_pe66.oe66 (.text:ti_sysbios_knl_Semaphore_Object__destruct__S)
                  8000b940    00000040     app_pe66.oe66 (.text:ti_sysbios_knl_Swi_Object__get__S)
                  8000b980    00000040     app_pe66.oe66 (.text:ti_sysbios_knl_Task_Object__get__S)
                  8000b9c0    00000040     sysbios.ae66 : BIOS.obj (.text:ti_sysbios_knl_Task_sleepTimeout__I)
                  8000ba00    00000040                  : BIOS.obj (.text:ti_sysbios_timers_dmtimer_Timer_stub__E)
                  8000ba40    00000040     ti.targets.rts6000.ae66 : Error.oe66 (.text:xdc_runtime_Error_check__E)
                  8000ba80    00000040                             : Error.oe66 (.text:xdc_runtime_Error_init__E)
                  8000bac0    00000040     app_pe66.oe66 (.text:xdc_runtime_LoggerBuf_Handle__label__S)
                  8000bb00    00000040     ti.targets.rts6000.ae66 : LoggerBuf.oe66 (.text:xdc_runtime_LoggerBuf_Instance_finalize__E)
                  8000bb40    00000040     app_pe66.oe66 (.text:xdc_runtime_LoggerBuf_Object__get__S)
                  8000bb80    00000040     ti.targets.rts6000.ae66 : LoggerBuf.oe66 (.text:xdc_runtime_LoggerBuf_reset__E)
                  8000bbc0    00000040                             : LoggerBuf.oe66 (.text:xdc_runtime_LoggerBuf_write0__E)
                  8000bc00    00000040                             : Memory.oe66 (.text:xdc_runtime_Memory_free__E)
                  8000bc40    00000040                             : Registry.oe66 (.text:xdc_runtime_Registry_findById__E)
                  8000bc80    00000040                             : System.oe66 (.text:xdc_runtime_System_abort__E)
                  8000bcc0    00000040     app_pe66.oe66 (.text:xdc_runtime_System_aprintf__E)
                  8000bd00    00000040     ti.targets.rts6000.ae66 : System.oe66 (.text:xdc_runtime_System_exit__E)
                  8000bd40    00000040     app_pe66.oe66 (.text:xdc_runtime_System_printf__E)
                  8000bd80    00000040     ti.targets.rts6000.ae66 : Text.oe66 (.text:xdc_runtime_Text_ropeText__E)
                  8000bdc0    00000020                             : LoggerBuf.oe66 (.text:LoggerBuf_instanceStartup)
                  8000bde0    00000020                             : xdc_noinit.oe66 (.text:__xdc__init)
                  8000be00    00000020     rts6600_elf.lib : _lock.obj (.text:_nop)
                  8000be20    00000020                     : _lock.obj (.text:_register_lock)
                  8000be40    00000020                     : _data_synch.obj (.text:_register_synch_api)
                  8000be60    00000020                     : _lock.obj (.text:_register_unlock)
                  8000be80    00000020     sysbios.ae66 : c62_TaskSupport_asm.obj (.text:_ti_sysbios_family_c62_TaskSupport_glue)
                  8000bea0    00000020     rts6600_elf.lib : exit.obj (.text:abort)
                  8000bec0    00000020                     : copy_zero_init.obj (.text:decompress:ZI:__TI_zero_init)
                  8000bee0    00000020                     : copy_decompress_none.obj (.text:decompress:none:__TI_decompress_none)
                  8000bf00    00000020                     : copy_decompress_rle.obj (.text:decompress:rle24:__TI_decompress_rle24)
                  8000bf20    00000020     app_pe66.oe66 (.text:ti_sysbios_BIOS_RtsGateProxy_enter__E)
                  8000bf40    00000020     app_pe66.oe66 (.text:ti_sysbios_BIOS_RtsGateProxy_leave__E)
                  8000bf60    00000020     sysbios.ae66 : BIOS.obj (.text:ti_sysbios_BIOS_exit__E)
                  8000bf80    00000020                  : BIOS.obj (.text:ti_sysbios_BIOS_getCpuFreq__E)
                  8000bfa0    00000020                  : BIOS.obj (.text:ti_sysbios_BIOS_linkedWithIncorrectBootLibrary__E)
                  8000bfc0    00000020     app_pe66.oe66 (.text:ti_sysbios_BIOS_nullFunc__I)
                  8000bfe0    00000020     sysbios.ae66 : BIOS.obj (.text:ti_sysbios_BIOS_setThreadType__E)
                  8000c000    00000020                  : BIOS.obj (.text:ti_sysbios_BIOS_start__E)
                  8000c020    00000020     app_pe66.oe66 (.text:ti_sysbios_family_c62_TaskSupport_Module__startupDone__S)
                  8000c040    00000020     sysbios.ae66 : BIOS.obj (.text:ti_sysbios_family_c62_TaskSupport_checkStack__E)
                  8000c060    00000020                  : BIOS.obj (.text:ti_sysbios_family_c62_TaskSupport_getStackAlignment__E)
                  8000c080    00000020     app_pe66.oe66 (.text:ti_sysbios_family_c64p_Hwi_Module__startupDone__F)
                  8000c0a0    00000020     sysbios.ae66 : BIOS.obj (.text:ti_sysbios_family_c64p_Hwi_clearInterrupt__E)
                  8000c0c0    00000020                  : BIOS.obj (.text:ti_sysbios_family_c64p_Hwi_startup__E)
                  8000c0e0    00000020                  : BIOS.obj (.text:ti_sysbios_family_c64p_Hwi_switchFromBootStack__E)
                  8000c100    00000020                  : BIOS.obj (.text:ti_sysbios_family_c64p_TimestampProvider_Module_startup__E)
                  8000c120    00000020                  : BIOS.obj (.text:ti_sysbios_family_c64p_TimestampProvider_get32__E)
                  8000c140    00000020                  : BIOS.obj (.text:ti_sysbios_family_c64p_TimestampProvider_get64__E)
                  8000c160    00000020                  : BIOS.obj (.text:ti_sysbios_family_c66_Cache_RTSSynchInv__I)
                  8000c180    00000020                  : BIOS.obj (.text:ti_sysbios_family_c66_Cache_RTSSynchWbInv__I)
                  8000c1a0    00000020                  : BIOS.obj (.text:ti_sysbios_family_c66_Cache_RTSSynchWb__I)
                  8000c1c0    00000020                  : BIOS.obj (.text:ti_sysbios_family_c66_Cache_wait__E)
                  8000c1e0    00000020     app_pe66.oe66 (.text:ti_sysbios_family_shared_vayu_TimerSupport_Module__startupDone__F)
                  8000c200    00000020     sysbios.ae66 : BIOS.obj (.text:ti_sysbios_family_shared_vayu_TimerSupport_Module_startup__E)
                  8000c220    00000020                  : BIOS.obj (.text:ti_sysbios_family_shared_vayu_TimerSupport_enable__E)
                  8000c240    00000020                  : BIOS.obj (.text:ti_sysbios_gates_GateHwi_Instance_init__E)
                  8000c260    00000020                  : BIOS.obj (.text:ti_sysbios_gates_GateHwi_enter__E)
                  8000c280    00000020                  : BIOS.obj (.text:ti_sysbios_gates_GateHwi_leave__E)
                  8000c2a0    00000020                  : BIOS.obj (.text:ti_sysbios_gates_GateHwi_query__E)
                  8000c2c0    00000020                  : BIOS.obj (.text:ti_sysbios_gates_GateMutex_Instance_finalize__E)
                  8000c2e0    00000020                  : BIOS.obj (.text:ti_sysbios_gates_GateMutex_query__E)
                  8000c300    00000020                  : BIOS.obj (.text:ti_sysbios_hal_Hwi_Module_startup__E)
                  8000c320    00000020     app_pe66.oe66 (.text:ti_sysbios_heaps_HeapMem_Module_GateProxy_enter__E)
                  8000c340    00000020     app_pe66.oe66 (.text:ti_sysbios_heaps_HeapMem_Module_GateProxy_leave__E)
                  8000c360    00000020     sysbios.ae66 : BIOS.obj (.text:ti_sysbios_heaps_HeapMem_isBlocking__E)
                  8000c380    00000020     app_pe66.oe66 (.text:ti_sysbios_knl_Clock_TimerProxy_getMaxTicks__E)
                  8000c3a0    00000020     sysbios.ae66 : BIOS.obj (.text:ti_sysbios_knl_Idle_loop__E)
                  8000c3c0    00000020                  : BIOS.obj (.text:ti_sysbios_knl_Queue_Instance_init__E)
                  8000c3e0    00000020     app_pe66.oe66 (.text:ti_sysbios_knl_Queue_Object__destruct__S)
                  8000c400    00000020     app_pe66.oe66 (.text:ti_sysbios_knl_Queue_Object__get__S)
                  8000c420    00000020     app_pe66.oe66 (.text:ti_sysbios_knl_Queue_destruct)
                  8000c440    00000020     sysbios.ae66 : BIOS.obj (.text:ti_sysbios_knl_Queue_empty__E)
                  8000c460    00000020                  : BIOS.obj (.text:ti_sysbios_knl_Semaphore_Instance_finalize__E)
                  8000c480    00000020     app_pe66.oe66 (.text:ti_sysbios_knl_Semaphore_destruct)
                  8000c4a0    00000020     sysbios.ae66 : BIOS.obj (.text:ti_sysbios_knl_Swi_disable__E)
                  8000c4c0    00000020                  : BIOS.obj (.text:ti_sysbios_knl_Task_disable__E)
                  8000c4e0    00000020                  : BIOS.obj (.text:ti_sysbios_knl_Task_startup__E)
                  8000c500    00000020     app_pe66.oe66 (.text:ti_sysbios_timers_dmtimer_Timer_Module__startupDone__F)
                  8000c520    00000020     sysbios.ae66 : BIOS.obj (.text:ti_sysbios_timers_dmtimer_Timer_getMaxTicks__E)
                  8000c540    00000020     ti.targets.rts6000.ae66 : Error.oe66 (.text:xdc_runtime_Error_getSite__E)
                  8000c560    00000020                             : Error.oe66 (.text:xdc_runtime_Error_raiseX__E)
                  8000c580    00000020                             : Gate.oe66 (.text:xdc_runtime_Gate_enterSystem__E)
                  8000c5a0    00000020                             : Gate.oe66 (.text:xdc_runtime_Gate_leaveSystem__E)
                  8000c5c0    00000020     app_pe66.oe66 (.text:xdc_runtime_IHeap_alloc)
                  8000c5e0    00000020     app_pe66.oe66 (.text:xdc_runtime_IHeap_free)
                  8000c600    00000020     app_pe66.oe66 (.text:xdc_runtime_LoggerBuf_Module_GateProxy_enter__E)
                  8000c620    00000020     app_pe66.oe66 (.text:xdc_runtime_LoggerBuf_Module_GateProxy_leave__E)
                  8000c640    00000020     ti.targets.rts6000.ae66 : LoggerBuf.oe66 (.text:xdc_runtime_LoggerBuf_disable__E)
                  8000c660    00000020                             : LoggerBuf.oe66 (.text:xdc_runtime_LoggerBuf_enable__E)
                  8000c680    00000020                             : LoggerBuf.oe66 (.text:xdc_runtime_LoggerBuf_write1__E)
                  8000c6a0    00000020                             : LoggerBuf.oe66 (.text:xdc_runtime_LoggerBuf_write2__E)
                  8000c6c0    00000020                             : Memory.oe66 (.text:xdc_runtime_Memory_calloc__E)
                  8000c6e0    00000020                             : Memory.oe66 (.text:xdc_runtime_Memory_getMaxDefaultTypeAlign__E)
                  8000c700    00000020     app_pe66.oe66 (.text:xdc_runtime_Startup_exec__I)
                  8000c720    00000020     ti.targets.rts6000.ae66 : Startup.oe66 (.text:xdc_runtime_Startup_rtsDone__E)
                  8000c740    00000020                             : SysMin.oe66 (.text:xdc_runtime_SysMin_ready__E)
                  8000c760    00000020     app_pe66.oe66 (.text:xdc_runtime_System_Module_GateProxy_enter__E)
                  8000c780    00000020     app_pe66.oe66 (.text:xdc_runtime_System_Module_GateProxy_leave__E)
                  8000c7a0    00000020     ti.targets.rts6000.ae66 : System.oe66 (.text:xdc_runtime_System_Module_startup__E)
                  8000c7c0    00000020                             : System.oe66 (.text:xdc_runtime_System_aprintf_va__F)
                  8000c7e0    00000020                             : System.oe66 (.text:xdc_runtime_System_printf_va__F)
                  8000c800    00000020                             : System.oe66 (.text:xdc_runtime_System_vsnprintf__E)
                  8000c820    00000020     app_pe66.oe66 (.text:xdc_runtime_Text_visitRope__I)

.const     0    8000c840    00002d8a     
                  8000c840    00001ca4     app_pe66.oe66 (.const:xdc_runtime_Text_charTab__A)
                  8000e4e4    00000518     sysbios.ae66 : BIOS.obj (.const:.string)
                  8000e9fc    00000004     ti.targets.rts6000.ae66 : Assert.oe66 (.const:.string)
                  8000ea00    00000400     app_pe66.oe66 (.const:ti_sysbios_family_c66_Cache_marvalues__C)
                  8000ee00    000000dc     app_pe66.oe66 (.const:xdc_runtime_Text_nodeTab__A)
                  8000eedc    00000064     app_pe66.oe66 (.const:.string)
                  8000ef40    00000058     ti.targets.rts6000.ae66 : Error.oe66 (.const:.string)
                  8000ef98    0000004c     main.obj (.const:.string)
                  8000efe4    00000040     ti.targets.rts6000.ae66 : Text.oe66 (.const:.string)
                  8000f024    0000003c     app_pe66.oe66 (.const:ti_sysbios_knl_Task_Object__PARAMS__C)
                  8000f060    0000003c     app_pe66.oe66 (.const:xdc_runtime_LoggerBuf_Module__FXNS__C)
                  8000f09c    00000004     app_pe66.oe66 (.const:ti_sysbios_family_c62_TaskSupport_stackAlignment__C)
                  8000f0a0    00000034     app_pe66.oe66 (.const:xdc_runtime_Startup_sfxnTab__A)
                  8000f0d4    0000002c     ti.targets.rts6000.ae66 : Startup.oe66 (.const:.string)
                  8000f100    00000028     app_pe66.oe66 (.const:ti_sysbios_heaps_HeapMem_Module__FXNS__C)
                  8000f128    00000028     app_pe66.oe66 (.const:xdc_runtime_LoggerBuf_Object__PARAMS__C)
                  8000f150    00000024     app_pe66.oe66 (.const:ti_sysbios_gates_GateHwi_Module__FXNS__C)
                  8000f174    00000024     app_pe66.oe66 (.const:ti_sysbios_gates_GateMutex_Module__FXNS__C)
                  8000f198    00000024     app_pe66.oe66 (.const:ti_sysbios_heaps_HeapMem_Object__PARAMS__C)
                  8000f1bc    00000024     app_pe66.oe66 (.const:ti_sysbios_knl_Semaphore_Object__PARAMS__C)
                  8000f1e0    00000020     app_pe66.oe66 (.const:ti_sysbios_gates_GateHwi_Object__DESC__C)
                  8000f200    00000020     app_pe66.oe66 (.const:ti_sysbios_gates_GateMutex_Object__DESC__C)
                  8000f220    00000020     app_pe66.oe66 (.const:ti_sysbios_heaps_HeapMem_Object__DESC__C)
                  8000f240    00000020     app_pe66.oe66 (.const:ti_sysbios_knl_Queue_Object__DESC__C)
                  8000f260    00000020     app_pe66.oe66 (.const:ti_sysbios_knl_Semaphore_Object__DESC__C)
                  8000f280    00000020     app_pe66.oe66 (.const:ti_sysbios_knl_Task_Object__DESC__C)
                  8000f2a0    00000020     app_pe66.oe66 (.const:xdc_runtime_LoggerBuf_Object__DESC__C)
                  8000f2c0    0000001a     app_pe66.oe66 (.const:xdc_runtime_Startup_sfxnRts__A)
                  8000f2da    00000002     app_pe66.oe66 (.const:ti_sysbios_family_c64p_Exception_Module__id__C)
                  8000f2dc    00000018     app_pe66.oe66 (.const:ti_sysbios_gates_GateHwi_Object__PARAMS__C)
                  8000f2f4    00000018     app_pe66.oe66 (.const:ti_sysbios_gates_GateMutex_Object__PARAMS__C)
                  8000f30c    00000018     app_pe66.oe66 (.const:ti_sysbios_knl_Queue_Object__PARAMS__C)
                  8000f324    00000004     app_pe66.oe66 (.const:ti_sysbios_family_c64p_Exception_E_exceptionMax__C)
                  8000f328    00000011     ti.targets.rts6000.ae66 : System.oe66 (.const:.string:digtohex)
                  8000f339    00000001     --HOLE-- [fill = 0]
                  8000f33a    00000002     app_pe66.oe66 (.const:ti_sysbios_family_c64p_Exception_useInternalBuffer__C)
                  8000f33c    00000008     ti.targets.rts6000.ae66 : System.oe66 (.const:.string)
                  8000f344    00000008     app_pe66.oe66 (.const:ti_sysbios_knl_Idle_funcList__C)
                  8000f34c    00000004     app_pe66.oe66 (.const:ti_sysbios_family_c64p_Exception_exceptionHook__C)
                  8000f350    00000008     app_pe66.oe66 (.const:xdc_runtime_Startup_firstFxns__A)
                  8000f358    00000008     app_pe66.oe66 (.const:xdc_runtime_Startup_firstFxns__C)
                  8000f360    00000008     app_pe66.oe66 (.const:xdc_runtime_Startup_lastFxns__C)
                  8000f368    00000004     app_pe66.oe66 (.const:ti_sysbios_family_c64p_Exception_externalHook__C)
                  8000f36c    00000004     app_pe66.oe66 (.const:ti_sysbios_family_c64p_Exception_internalHook__C)
                  8000f370    00000004     app_pe66.oe66 (.const:ti_sysbios_family_c64p_Exception_nmiHook__C)
                  8000f374    00000004     app_pe66.oe66 (.const:ti_sysbios_family_c64p_Hwi_LD_end__C)
                  8000f378    00000004     app_pe66.oe66 (.const:ti_sysbios_family_c64p_Hwi_LM_begin__C)
                  8000f37c    00000004     app_pe66.oe66 (.const:ti_sysbios_family_c64p_Hwi_Module__diagsEnabled__C)
                  8000f380    00000004     app_pe66.oe66 (.const:ti_sysbios_family_c64p_Hwi_Module__diagsIncluded__C)
                  8000f384    00000004     app_pe66.oe66 (.const:ti_sysbios_family_c64p_Hwi_Module__diagsMask__C)
                  8000f388    00000004     app_pe66.oe66 (.const:ti_sysbios_family_c64p_Hwi_Module__loggerFxn1__C)
                  8000f38c    00000004     app_pe66.oe66 (.const:ti_sysbios_family_c64p_Hwi_Module__loggerFxn8__C)
                  8000f390    00000004     app_pe66.oe66 (.const:ti_sysbios_family_c64p_Hwi_Module__loggerObj__C)
                  8000f394    00000004     app_pe66.oe66 (.const:ti_sysbios_family_c66_Cache_E_invalidL1CacheSize__C)
                  8000f398    00000004     app_pe66.oe66 (.const:ti_sysbios_family_c66_Cache_E_invalidL2CacheSize__C)
                  8000f39c    00000004     app_pe66.oe66 (.const:ti_sysbios_family_c66_Cache_atomicBlockSize__C)
                  8000f3a0    00000004     app_pe66.oe66 (.const:ti_sysbios_gates_GateMutex_A_badContext__C)
                  8000f3a4    00000004     app_pe66.oe66 (.const:ti_sysbios_gates_GateMutex_Instance_State_sem__O)
                  8000f3a8    00000004     app_pe66.oe66 (.const:ti_sysbios_gates_GateMutex_Module__diagsEnabled__C)
                  8000f3ac    00000004     app_pe66.oe66 (.const:ti_sysbios_gates_GateMutex_Module__diagsIncluded__C)
                  8000f3b0    00000004     app_pe66.oe66 (.const:ti_sysbios_gates_GateMutex_Module__diagsMask__C)
                  8000f3b4    00000004     app_pe66.oe66 (.const:ti_sysbios_hal_Hwi_E_stackOverflow__C)
                  8000f3b8    00000004     app_pe66.oe66 (.const:ti_sysbios_heaps_HeapMem_A_align__C)
                  8000f3bc    00000004     app_pe66.oe66 (.const:ti_sysbios_heaps_HeapMem_A_heapSize__C)
                  8000f3c0    00000004     app_pe66.oe66 (.const:ti_sysbios_heaps_HeapMem_A_invalidFree__C)
                  8000f3c4    00000004     app_pe66.oe66 (.const:ti_sysbios_heaps_HeapMem_A_zeroBlock__C)
                  8000f3c8    00000004     app_pe66.oe66 (.const:ti_sysbios_heaps_HeapMem_E_memory__C)
                  8000f3cc    00000004     app_pe66.oe66 (.const:ti_sysbios_heaps_HeapMem_Module__diagsEnabled__C)
                  8000f3d0    00000004     app_pe66.oe66 (.const:ti_sysbios_heaps_HeapMem_Module__diagsIncluded__C)
                  8000f3d4    00000004     app_pe66.oe66 (.const:ti_sysbios_heaps_HeapMem_Module__diagsMask__C)
                  8000f3d8    00000004     app_pe66.oe66 (.const:ti_sysbios_heaps_HeapMem_Module__gateObj__C)
                  8000f3dc    00000004     app_pe66.oe66 (.const:ti_sysbios_heaps_HeapMem_Object__count__C)
                  8000f3e0    00000004     app_pe66.oe66 (.const:ti_sysbios_heaps_HeapMem_reqAlign__C)
                  8000f3e4    00000004     app_pe66.oe66 (.const:ti_sysbios_knl_Clock_LM_begin__C)
                  8000f3e8    00000004     app_pe66.oe66 (.const:ti_sysbios_knl_Clock_LM_tick__C)
                  8000f3ec    00000004     app_pe66.oe66 (.const:ti_sysbios_knl_Clock_LW_delayed__C)
                  8000f3f0    00000004     app_pe66.oe66 (.const:ti_sysbios_knl_Clock_Module_State_clockQ__O)
                  8000f3f4    00000004     app_pe66.oe66 (.const:ti_sysbios_knl_Clock_Module__diagsEnabled__C)
                  8000f3f8    00000004     app_pe66.oe66 (.const:ti_sysbios_knl_Clock_Module__diagsIncluded__C)
                  8000f3fc    00000004     app_pe66.oe66 (.const:ti_sysbios_knl_Clock_Module__diagsMask__C)
                  8000f400    00000004     app_pe66.oe66 (.const:ti_sysbios_knl_Clock_Module__loggerFxn1__C)
                  8000f404    00000004     app_pe66.oe66 (.const:ti_sysbios_knl_Clock_Module__loggerFxn2__C)
                  8000f408    00000004     app_pe66.oe66 (.const:ti_sysbios_knl_Clock_Module__loggerObj__C)
                  8000f40c    00000004     app_pe66.oe66 (.const:ti_sysbios_knl_Semaphore_A_badContext__C)
                  8000f410    00000004     app_pe66.oe66 (.const:ti_sysbios_knl_Idle_funcList__A)
                  8000f414    00000004     app_pe66.oe66 (.const:ti_sysbios_knl_Semaphore_A_noEvents__C)
                  8000f418    00000004     app_pe66.oe66 (.const:ti_sysbios_knl_Semaphore_A_overflow__C)
                  8000f41c    00000004     app_pe66.oe66 (.const:ti_sysbios_knl_Semaphore_A_pendTaskDisabled__C)
                  8000f420    00000004     app_pe66.oe66 (.const:ti_sysbios_knl_Semaphore_Instance_State_pendQ__O)
                  8000f424    00000004     app_pe66.oe66 (.const:ti_sysbios_knl_Semaphore_LM_pend__C)
                  8000f428    00000004     app_pe66.oe66 (.const:ti_sysbios_knl_Semaphore_LM_post__C)
                  8000f42c    00000004     app_pe66.oe66 (.const:ti_sysbios_knl_Semaphore_Module__diagsEnabled__C)
                  8000f430    00000004     app_pe66.oe66 (.const:ti_sysbios_knl_Semaphore_Module__diagsIncluded__C)
                  8000f434    00000004     app_pe66.oe66 (.const:ti_sysbios_knl_Semaphore_Module__diagsMask__C)
                  8000f438    00000004     app_pe66.oe66 (.const:ti_sysbios_knl_Semaphore_Module__loggerFxn2__C)
                  8000f43c    00000004     app_pe66.oe66 (.const:ti_sysbios_knl_Semaphore_Module__loggerFxn4__C)
                  8000f440    00000004     app_pe66.oe66 (.const:ti_sysbios_knl_Semaphore_Module__loggerObj__C)
                  8000f444    00000004     app_pe66.oe66 (.const:ti_sysbios_knl_Swi_LD_end__C)
                  8000f448    00000004     app_pe66.oe66 (.const:ti_sysbios_knl_Swi_LM_begin__C)
                  8000f44c    00000004     app_pe66.oe66 (.const:ti_sysbios_knl_Swi_LM_post__C)
                  8000f450    00000004     app_pe66.oe66 (.const:ti_sysbios_knl_Swi_Module__diagsEnabled__C)
                  8000f454    00000004     app_pe66.oe66 (.const:ti_sysbios_knl_Swi_Module__diagsIncluded__C)
                  8000f458    00000004     app_pe66.oe66 (.const:ti_sysbios_knl_Swi_Module__diagsMask__C)
                  8000f45c    00000004     app_pe66.oe66 (.const:ti_sysbios_knl_Swi_Module__loggerFxn1__C)
                  8000f460    00000004     app_pe66.oe66 (.const:ti_sysbios_knl_Swi_Module__loggerFxn4__C)
                  8000f464    00000004     app_pe66.oe66 (.const:ti_sysbios_knl_Swi_Module__loggerObj__C)
                  8000f468    00000004     app_pe66.oe66 (.const:ti_sysbios_knl_Swi_Object__count__C)
                  8000f46c    00000004     app_pe66.oe66 (.const:ti_sysbios_knl_Task_A_badPriority__C)
                  8000f470    00000004     app_pe66.oe66 (.const:ti_sysbios_knl_Task_A_badTaskState__C)
                  8000f474    00000004     app_pe66.oe66 (.const:ti_sysbios_knl_Task_A_badThreadType__C)
                  8000f478    00000004     app_pe66.oe66 (.const:ti_sysbios_knl_Task_A_badTimeout__C)
                  8000f47c    00000004     app_pe66.oe66 (.const:ti_sysbios_knl_Task_A_noPendElem__C)
                  8000f480    00000004     app_pe66.oe66 (.const:ti_sysbios_knl_Task_A_sleepTaskDisabled__C)
                  8000f484    00000004     app_pe66.oe66 (.const:ti_sysbios_knl_Task_E_spOutOfBounds__C)
                  8000f488    00000004     app_pe66.oe66 (.const:ti_sysbios_knl_Task_E_stackOverflow__C)
                  8000f48c    00000004     app_pe66.oe66 (.const:ti_sysbios_knl_Task_LD_block__C)
                  8000f490    00000004     app_pe66.oe66 (.const:ti_sysbios_knl_Task_LD_exit__C)
                  8000f494    00000004     app_pe66.oe66 (.const:ti_sysbios_knl_Task_LD_ready__C)
                  8000f498    00000004     app_pe66.oe66 (.const:ti_sysbios_knl_Task_LM_sleep__C)
                  8000f49c    00000004     app_pe66.oe66 (.const:ti_sysbios_knl_Task_LM_switch__C)
                  8000f4a0    00000004     app_pe66.oe66 (.const:ti_sysbios_knl_Task_Module_State_inactiveQ__O)
                  8000f4a4    00000004     app_pe66.oe66 (.const:ti_sysbios_knl_Task_Module__diagsEnabled__C)
                  8000f4a8    00000004     app_pe66.oe66 (.const:ti_sysbios_knl_Task_Module__diagsIncluded__C)
                  8000f4ac    00000004     app_pe66.oe66 (.const:ti_sysbios_knl_Task_Module__diagsMask__C)
                  8000f4b0    00000004     app_pe66.oe66 (.const:ti_sysbios_knl_Task_Module__loggerFxn2__C)
                  8000f4b4    00000004     app_pe66.oe66 (.const:ti_sysbios_knl_Task_Module__loggerFxn4__C)
                  8000f4b8    00000004     app_pe66.oe66 (.const:ti_sysbios_knl_Task_Module__loggerObj__C)
                  8000f4bc    00000004     app_pe66.oe66 (.const:ti_sysbios_knl_Task_Object__count__C)
                  8000f4c0    00000004     app_pe66.oe66 (.const:ti_sysbios_knl_Task_allBlockedFunc__C)
                  8000f4c4    00000004     app_pe66.oe66 (.const:ti_sysbios_knl_Task_defaultStackHeap__C)
                  8000f4c8    00000004     app_pe66.oe66 (.const:ti_sysbios_knl_Task_defaultStackSize__C)
                  8000f4cc    00000004     app_pe66.oe66 (.const:ti_sysbios_knl_Task_numConstructedTasks__C)
                  8000f4d0    00000004     app_pe66.oe66 (.const:ti_sysbios_timers_dmtimer_Timer_E_cannotSupport__C)
                  8000f4d4    00000004     app_pe66.oe66 (.const:ti_sysbios_timers_dmtimer_Timer_E_freqMismatch__C)
                  8000f4d8    00000004     app_pe66.oe66 (.const:ti_sysbios_timers_dmtimer_Timer_Module__diagsEnabled__C)
                  8000f4dc    00000004     app_pe66.oe66 (.const:ti_sysbios_timers_dmtimer_Timer_Module__diagsIncluded__C)
                  8000f4e0    00000004     app_pe66.oe66 (.const:ti_sysbios_timers_dmtimer_Timer_Module__diagsMask__C)
                  8000f4e4    00000004     app_pe66.oe66 (.const:ti_sysbios_timers_dmtimer_Timer_numTimerDevices__C)
                  8000f4e8    00000004     app_pe66.oe66 (.const:xdc_runtime_Assert_E_assertFailed__C)
                  8000f4ec    00000004     app_pe66.oe66 (.const:xdc_runtime_Core_A_initializedParams__C)
                  8000f4f0    00000004     app_pe66.oe66 (.const:xdc_runtime_Core_Module__diagsEnabled__C)
                  8000f4f4    00000004     app_pe66.oe66 (.const:xdc_runtime_Core_Module__diagsIncluded__C)
                  8000f4f8    00000004     app_pe66.oe66 (.const:xdc_runtime_Core_Module__diagsMask__C)
                  8000f4fc    00000004     app_pe66.oe66 (.const:xdc_runtime_Error_E_memory__C)
                  8000f500    00000004     app_pe66.oe66 (.const:xdc_runtime_Error_Module__diagsEnabled__C)
                  8000f504    00000004     app_pe66.oe66 (.const:xdc_runtime_Error_Module__diagsIncluded__C)
                  8000f508    00000004     app_pe66.oe66 (.const:xdc_runtime_Error_Module__diagsMask__C)
                  8000f50c    00000004     app_pe66.oe66 (.const:xdc_runtime_Error_Module__loggerFxn8__C)
                  8000f510    00000004     app_pe66.oe66 (.const:xdc_runtime_Error_Module__loggerObj__C)
                  8000f514    00000004     app_pe66.oe66 (.const:xdc_runtime_Error_policyFxn__C)
                  8000f518    00000004     app_pe66.oe66 (.const:xdc_runtime_Error_policy__C)
                  8000f51c    00000004     app_pe66.oe66 (.const:xdc_runtime_Error_raiseHook__C)
                  8000f520    00000004     app_pe66.oe66 (.const:xdc_runtime_IFilterLogger_Interface__BASE__C)
                  8000f524    00000004     app_pe66.oe66 (.const:xdc_runtime_IGateProvider_Interface__BASE__C)
                  8000f528    00000004     app_pe66.oe66 (.const:xdc_runtime_IHeap_Interface__BASE__C)
                  8000f52c    00000004     app_pe66.oe66 (.const:xdc_runtime_ILogger_Interface__BASE__C)
                  8000f530    00000004     app_pe66.oe66 (.const:xdc_runtime_IModule_Interface__BASE__C)
                  8000f534    00000004     app_pe66.oe66 (.const:xdc_runtime_Log_L_error__C)
                  8000f538    00000004     app_pe66.oe66 (.const:xdc_runtime_LoggerBuf_E_badLevel__C)
                  8000f53c    00000004     app_pe66.oe66 (.const:xdc_runtime_LoggerBuf_Module__gateObj__C)
                  8000f540    00000004     app_pe66.oe66 (.const:xdc_runtime_LoggerBuf_Object__count__C)
                  8000f544    00000004     app_pe66.oe66 (.const:xdc_runtime_LoggerBuf_statusLogger__C)
                  8000f548    00000004     app_pe66.oe66 (.const:xdc_runtime_Memory_defaultHeapInstance__C)
                  8000f54c    00000004     app_pe66.oe66 (.const:xdc_runtime_Startup_execImpl__C)
                  8000f550    00000004     app_pe66.oe66 (.const:xdc_runtime_Startup_maxPasses__C)
                  8000f554    00000004     app_pe66.oe66 (.const:xdc_runtime_Startup_sfxnRts__C)
                  8000f558    00000004     app_pe66.oe66 (.const:xdc_runtime_Startup_sfxnTab__C)
                  8000f55c    00000004     app_pe66.oe66 (.const:xdc_runtime_SysMin_bufSize__C)
                  8000f560    00000004     app_pe66.oe66 (.const:xdc_runtime_SysMin_outputFunc__C)
                  8000f564    00000004     app_pe66.oe66 (.const:xdc_runtime_System_Module__gateObj__C)
                  8000f568    00000004     app_pe66.oe66 (.const:xdc_runtime_System_abortFxn__C)
                  8000f56c    00000004     app_pe66.oe66 (.const:xdc_runtime_System_exitFxn__C)
                  8000f570    00000004     app_pe66.oe66 (.const:xdc_runtime_System_extendFxn__C)
                  8000f574    00000004     app_pe66.oe66 (.const:xdc_runtime_System_maxAtexitHandlers__C)
                  8000f578    00000004     app_pe66.oe66 (.const:xdc_runtime_Text_charTab__C)
                  8000f57c    00000004     app_pe66.oe66 (.const:xdc_runtime_Text_nameEmpty__C)
                  8000f580    00000004     app_pe66.oe66 (.const:xdc_runtime_Text_nameStatic__C)
                  8000f584    00000004     app_pe66.oe66 (.const:xdc_runtime_Text_nameUnknown__C)
                  8000f588    00000004     app_pe66.oe66 (.const:xdc_runtime_Text_nodeTab__C)
                  8000f58c    00000004     app_pe66.oe66 (.const:xdc_runtime_Text_visitRopeFxn__C)
                  8000f590    00000002     app_pe66.oe66 (.const:ti_sysbios_family_c64p_Hwi_Module__id__C)
                  8000f592    00000002     app_pe66.oe66 (.const:ti_sysbios_family_c64p_Hwi_Module__loggerDefined__C)
                  8000f594    00000002     app_pe66.oe66 (.const:ti_sysbios_family_c66_Cache_Module__id__C)
                  8000f596    00000002     app_pe66.oe66 (.const:ti_sysbios_family_c66_Cache_registerRTSSynch__C)
                  8000f598    00000002     app_pe66.oe66 (.const:ti_sysbios_gates_GateMutex_Module__id__C)
                  8000f59a    00000002     app_pe66.oe66 (.const:ti_sysbios_hal_Hwi_Module__id__C)
                  8000f59c    00000002     app_pe66.oe66 (.const:ti_sysbios_heaps_HeapMem_Module__id__C)
                  8000f59e    00000002     app_pe66.oe66 (.const:ti_sysbios_knl_Clock_Module__id__C)
                  8000f5a0    00000002     app_pe66.oe66 (.const:ti_sysbios_knl_Clock_Module__loggerDefined__C)
                  8000f5a2    00000002     app_pe66.oe66 (.const:ti_sysbios_knl_Semaphore_Module__id__C)
                  8000f5a4    00000002     app_pe66.oe66 (.const:ti_sysbios_knl_Semaphore_Module__loggerDefined__C)
                  8000f5a6    00000002     app_pe66.oe66 (.const:ti_sysbios_knl_Swi_Module__id__C)
                  8000f5a8    00000002     app_pe66.oe66 (.const:ti_sysbios_knl_Swi_Module__loggerDefined__C)
                  8000f5aa    00000002     app_pe66.oe66 (.const:ti_sysbios_knl_Task_Module__id__C)
                  8000f5ac    00000002     app_pe66.oe66 (.const:ti_sysbios_knl_Task_Module__loggerDefined__C)
                  8000f5ae    00000002     app_pe66.oe66 (.const:ti_sysbios_timers_dmtimer_Timer_Module__id__C)
                  8000f5b0    00000002     app_pe66.oe66 (.const:ti_sysbios_timers_dmtimer_Timer_checkFrequency__C)
                  8000f5b2    00000002     app_pe66.oe66 (.const:ti_sysbios_timers_dmtimer_Timer_startupNeeded__C)
                  8000f5b4    00000002     app_pe66.oe66 (.const:xdc_runtime_Core_Module__id__C)
                  8000f5b6    00000002     app_pe66.oe66 (.const:xdc_runtime_Error_Module__loggerDefined__C)
                  8000f5b8    00000002     app_pe66.oe66 (.const:xdc_runtime_Error_maxDepth__C)
                  8000f5ba    00000002     app_pe66.oe66 (.const:xdc_runtime_LoggerBuf_Module__id__C)
                  8000f5bc    00000002     app_pe66.oe66 (.const:xdc_runtime_LoggerBuf_filterByLevel__C)
                  8000f5be    00000002     app_pe66.oe66 (.const:xdc_runtime_Memory_Module__id__C)
                  8000f5c0    00000002     app_pe66.oe66 (.const:xdc_runtime_SysMin_flushAtExit__C)
                  8000f5c2    00000002     app_pe66.oe66 (.const:xdc_runtime_Text_charCnt__C)
                  8000f5c4    00000002     app_pe66.oe66 (.const:xdc_runtime_Text_isLoaded__C)
                  8000f5c6    00000002     app_pe66.oe66 (.const:xdc_runtime_Text_registryModsLastId__C)
                  8000f5c8    00000002     app_pe66.oe66 (.const:xdc_runtime_Text_unnamedModsLastId__C)

.far       0    800115d0    00001c08     UNINITIALIZED
                  800115d0    00001000     (.common:ti_sysbios_heaps_HeapMem_Instance_State_0_buf__A)
                  800125d0    00000800     app_pe66.oe66 (.far:taskStackSection)
                  80012dd0    00000200     (.common:xdc_runtime_LoggerBuf_Instance_State_0_entryArr__A)
                  80012fd0    00000200     (.common:xdc_runtime_SysMin_Module_State_0_outbuf__A)
                  800131d0    00000008     (.common:parmbuf)

.fardata   0    800131d8    0000063c     UNINITIALIZED
                  800131d8    0000020c     app_pe66.oe66 (.fardata)
                  800133e4    00000004     rts6600_elf.lib : _lock.obj (.fardata:_lock)
                  800133e8    000000c0     app_pe66.oe66 (.fardata:ti_sysbios_timers_dmtimer_Timer_Module_State_0_device__A)
                  800134a8    00000080     app_pe66.oe66 (.fardata:ti_sysbios_knl_Swi_Module_State_0_readyQ__A)
                  80013528    00000080     app_pe66.oe66 (.fardata:ti_sysbios_knl_Task_Module_State_0_readyQ__A)
                  800135a8    00000080     app_pe66.oe66 (.fardata:ti_sysbios_timers_dmtimer_Timer_Module_State_0_intFreqs__A)
                  80013628    00000060     app_pe66.oe66 (.fardata:ti_sysbios_timers_dmtimer_Timer_Object__table__V)
                  80013688    0000004c     app_pe66.oe66 (.fardata:ti_sysbios_knl_Task_Object__table__V)
                  800136d4    00000004     rts6600_elf.lib : _lock.obj (.fardata:_unlock)
                  800136d8    00000040     app_pe66.oe66 (.fardata:ti_sysbios_gates_GateMutex_Object__table__V)
                  80013718    00000040     app_pe66.oe66 (.fardata:ti_sysbios_timers_dmtimer_Timer_Module_State_0_handles__A)
                  80013758    00000030     app_pe66.oe66 (.fardata:ti_sysbios_knl_Swi_Object__table__V)
                  80013788    00000024     app_pe66.oe66 (.fardata:xdc_runtime_LoggerBuf_Object__table__V)
                  800137ac    00000004     --HOLE--
                  800137b0    00000018     app_pe66.oe66 (.fardata:ti_sysbios_family_c64p_Hwi_Object__table__V)
                  800137c8    00000018     app_pe66.oe66 (.fardata:ti_sysbios_heaps_HeapMem_Object__table__V)
                  800137e0    00000010     app_pe66.oe66 (.fardata:xdc_runtime_System_Module_State_0_atexitHandlers__A)
                  800137f0    0000000c     rts6600_elf.lib : exit.obj (.fardata)
                  800137fc    00000004     --HOLE--
                  80013800    00000008     app_pe66.oe66 (.fardata:ti_sysbios_hal_Hwi_Object__table__V)
                  80013808    00000004     app_pe66.oe66 (.fardata:ti_sysbios_gates_GateHwi_Object__table__V)
                  8001380c    00000004     --HOLE--
                  80013810    00000004     app_pe66.oe66 (.fardata:ti_sysbios_knl_Task_Module_State_0_idleTask__A)

.cio       0    80013818    00000120     UNINITIALIZED
                  80013818    00000120     rts6600_elf.lib : trgmsg.obj (.cio)

.vecs      0    80013c00    00000200     
                  80013c00    00000200     app_pe66.oe66 (.vecs)

xdc.meta   0    80000000    00000100     COPY SECTION
                  80000000    00000100     app_pe66.oe66 (xdc.meta)

MODULE SUMMARY

       Module                     code    ro data   rw data
       ------                     ----    -------   -------
    .\
       main.obj                   192     76        0      
    +--+--------------------------+-------+---------+---------+
       Total:                     192     76        0      
                                                           
    C:\Users\a0282268\Documents\TI\Customer\ZTE\am5726\Test_bios\Debug\configPkg\package\cfg\
       app_pe66.oe66              4736    10052     8732   
    +--+--------------------------+-------+---------+---------+
       Total:                     4736    10052     8732   
                                                           
    C:\Users\a0282268\Documents\TI\Customer\ZTE\am5726\Test_bios\src\sysbios\sysbios.ae66
       BIOS.obj                   29920   1304      0      
       c64p_Hwi_disp_always.obj   512     0         0      
       c64p_Exception_asm.obj     384     0         0      
       c62_TaskSupport_asm.obj    224     0         0      
       c64p_Hwi_asm_switch.obj    192     0         0      
    +--+--------------------------+-------+---------+---------+
       Total:                     31232   1304      0      
                                                           
    C:\ti\bios_6_46_04_53\packages\ti\targets\rts6000\lib\boot.ae66
       autoinit.oe66              320     0         0      
       boot.oe66                  160     0         0      
    +--+--------------------------+-------+---------+---------+
       Total:                     480     0         0      
                                                           
    C:\ti\bios_6_46_04_53\packages\ti\targets\rts6000\lib\ti.targets.rts6000.ae66
       System.oe66                3200    25        0      
       LoggerBuf.oe66             2368    0         0      
       Text.oe66                  1696    64        0      
       Error.oe66                 1056    88        0      
       Core-mem.oe66              832     0         0      
       Startup.oe66               768     44        0      
       SysMin.oe66                704     0         0      
       Memory.oe66                448     0         0      
       Core-smem.oe66             384     0         0      
       Assert.oe66                160     4         0      
       Core-label.oe66            128     0         0      
       Core-params.oe66           128     0         0      
       Gate.oe66                  64      0         0      
       Registry.oe66              64      0         0      
       xdc_noinit.oe66            32      0         0      
    +--+--------------------------+-------+---------+---------+
       Total:                     12032   225       0      
                                                           
    C:\ti\ti-cgt-c6000_8.1.4\lib\rts6600_elf.lib
       imath64.obj                640     0         0      
       trgmsg.obj                 256     0         288    
       copy_decompress_rle.obj    288     0         0      
       exit.obj                   224     0         12     
       trgdrv.obj                 224     0         8      
       llshift.obj                224     0         0      
       memset.obj                 224     0         0      
       divu.obj                   192     0         0      
       tls.obj                    192     0         0      
       memcpy64.obj               160     0         0      
       remu.obj                   160     0         0      
       _lock.obj                  96      0         8      
       args_main.obj              64      0         0      
       strasg.obj                 64      0         0      
       _data_synch.obj            32      0         0      
       copy_decompress_none.obj   32      0         0      
       copy_zero_init.obj         32      0         0      
    +--+--------------------------+-------+---------+---------+
       Total:                     3104    0         316    
                                                           
       Stack:                     0       0         8192   
       Linker Generated:          0       1120      0      
    +--+--------------------------+-------+---------+---------+
       Grand Total:               51776   12777     17240  


LINKER GENERATED COPY TABLES

__TI_cinit_table @ 80014250 records: 2, size/record: 8, table size: 16
	.fardata: load addr=80013e00, load size=0000043c bytes, run addr=800131d8, run size=0000063c bytes, compression=rle
	.far: load addr=80014248, load size=00000008 bytes, run addr=800115d0, run size=00001c08 bytes, compression=zero_init


LINKER GENERATED HANDLER TABLE

__TI_handler_table @ 8001423c records: 3, size/record: 4, table size: 12
	index: 0, handler: __TI_decompress_rle24
	index: 1, handler: __TI_decompress_none
	index: 2, handler: __TI_zero_init


GLOBAL SYMBOLS: SORTED ALPHABETICALLY BY Name 

address   name                                                                    
-------   ----                                                                    
8000bea0  C$$EXIT                                                                 
8000a060  C$$IO$$                                                                 
80008780  HOSTwrite                                                               
8000bdc0  LoggerBuf_instanceStartup                                               
80000000  __ASM__                                                                 
80013818  __CIOBUF_                                                               
80000070  __ISA__                                                                 
80000088  __PLAT__                                                                
800000b0  __TARG__                                                                
80014250  __TI_CINIT_Base                                                         
80014260  __TI_CINIT_Limit                                                        
8001423c  __TI_Handler_Table_Base                                                 
80014248  __TI_Handler_Table_Limit                                                
UNDEFED   __TI_INITARRAY_Base                                                     
UNDEFED   __TI_INITARRAY_Limit                                                    
800115d0  __TI_STACK_END                                                          
00002000  __TI_STACK_SIZE                                                         
00000000  __TI_STATIC_BASE                                                        
UNDEFED   __TI_TLS_INIT_Base                                                      
UNDEFED   __TI_TLS_INIT_Limit                                                     
800137f0  __TI_cleanup_ptr                                                        
8000bee0  __TI_decompress_none                                                    
8000bf00  __TI_decompress_rle24                                                   
800137f4  __TI_dtors_ptr                                                          
800137f8  __TI_enable_exit_profile_output                                         
ffffffff  __TI_pprof_out_hndl                                                     
ffffffff  __TI_prof_data_size                                                     
ffffffff  __TI_prof_data_start                                                    
80009f80  __TI_readmsg                                                            
80009540  __TI_tls_init                                                           
8000a000  __TI_writemsg                                                           
8000bec0  __TI_zero_init                                                          
800000d8  __TRDR__                                                                
ffffffff  __binit__                                                               
80008e80  __c6xabi_divu                                                           
80004a80  __c6xabi_divull                                                         
8000a080  __c6xabi_llshl                                                          
8000ac80  __c6xabi_llshru                                                         
800096c0  __c6xabi_remu                                                           
8000b4c0  __c6xabi_strasgi_64plus                                                 
ffffffff  __c_args__                                                              
80008e80  __divu                                                                  
800096c0  __remu                                                                  
8000b4c0  __strasgi_64plus                                                        
8000bde0  __xdc__init                                                             
800133e0  __xdc__init__addr                                                       
8000b500  _args_main                                                              
00000000  _argsize                                                                
800071e0  _auto_init_elf                                                          
80009760  _c_int00                                                                
800133e4  _lock                                                                   
8000be00  _nop                                                                    
8000be20  _register_lock                                                          
8000be40  _register_synch_api                                                     
8000be60  _register_unlock                                                        
8000f5d0  _stack                                                                  
8000b540  _subcull                                                                
800136d4  _unlock                                                                 
8000bea0  abort                                                                   
ffffffff  binit                                                                   
80008f40  exit                                                                    
80009044  main                                                                    
80009800  memcpy                                                                  
80008860  memset                                                                  
80009000  taskFxn                                                                 
800131d8  ti_sysbios_BIOS_Module__state__V                                        
8000b780  ti_sysbios_BIOS_RtsGateProxy_Handle__label__S                           
8000af80  ti_sysbios_BIOS_RtsGateProxy_Object__delete__S                          
8000bf20  ti_sysbios_BIOS_RtsGateProxy_enter__E                                   
8000bf40  ti_sysbios_BIOS_RtsGateProxy_leave__E                                   
8000c2e0  ti_sysbios_BIOS_RtsGateProxy_query__E                                   
8000a180  ti_sysbios_BIOS_atExitFunc__I                                           
8000ada0  ti_sysbios_BIOS_errorRaiseHook__I                                       
8000b5c0  ti_sysbios_BIOS_exitFunc__I                                             
8000bf60  ti_sysbios_BIOS_exit__E                                                 
8000bf80  ti_sysbios_BIOS_getCpuFreq__E                                           
8000bfa0  ti_sysbios_BIOS_linkedWithIncorrectBootLibrary__E                       
8000bfc0  ti_sysbios_BIOS_nullFunc__I                                             
8000a200  ti_sysbios_BIOS_registerRTSLock__I                                      
8000ae00  ti_sysbios_BIOS_removeRTSLock__I                                        
8000b600  ti_sysbios_BIOS_rtsLock__I                                              
8000b640  ti_sysbios_BIOS_rtsUnlock__I                                            
8000bfe0  ti_sysbios_BIOS_setThreadType__E                                        
8000ae60  ti_sysbios_BIOS_startFunc__I                                            
8000c000  ti_sysbios_BIOS_start__E                                                
8000c020  ti_sysbios_family_c62_TaskSupport_Module__startupDone__S                
8000b580  ti_sysbios_family_c62_TaskSupport_buildTaskStack                        
8000c040  ti_sysbios_family_c62_TaskSupport_checkStack__E                         
8000c060  ti_sysbios_family_c62_TaskSupport_getStackAlignment__E                  
8000be80  ti_sysbios_family_c62_TaskSupport_glue                                  
8000f09c  ti_sysbios_family_c62_TaskSupport_stackAlignment__C                     
8000aec0  ti_sysbios_family_c62_TaskSupport_start__E                              
8000a100  ti_sysbios_family_c62_TaskSupport_swap__E                               
8000f324  ti_sysbios_family_c64p_Exception_E_exceptionMax__C                      
8000f2da  ti_sysbios_family_c64p_Exception_Module__id__C                          
800131fc  ti_sysbios_family_c64p_Exception_Module__state__V                       
800098a0  ti_sysbios_family_c64p_Exception_Module_startup__E                      
800067a0  ti_sysbios_family_c64p_Exception_dispatch__E                            
8000f34c  ti_sysbios_family_c64p_Exception_exceptionHook__C                       
8000f368  ti_sysbios_family_c64p_Exception_externalHook__C                        
80001060  ti_sysbios_family_c64p_Exception_handler__I                             
80004cc0  ti_sysbios_family_c64p_Exception_internalHandler__I                     
8000f36c  ti_sysbios_family_c64p_Exception_internalHook__C                        
8000f370  ti_sysbios_family_c64p_Exception_nmiHook__C                             
8000f33a  ti_sysbios_family_c64p_Exception_useInternalBuffer__C                   
80013c00  ti_sysbios_family_c64p_Hwi0                                             
8000f374  ti_sysbios_family_c64p_Hwi_LD_end__C                                    
8000f378  ti_sysbios_family_c64p_Hwi_LM_begin__C                                  
8000f37c  ti_sysbios_family_c64p_Hwi_Module__diagsEnabled__C                      
8000f380  ti_sysbios_family_c64p_Hwi_Module__diagsIncluded__C                     
8000f384  ti_sysbios_family_c64p_Hwi_Module__diagsMask__C                         
8000f590  ti_sysbios_family_c64p_Hwi_Module__id__C                                
8000f592  ti_sysbios_family_c64p_Hwi_Module__loggerDefined__C                     
8000f388  ti_sysbios_family_c64p_Hwi_Module__loggerFxn1__C                        
8000f38c  ti_sysbios_family_c64p_Hwi_Module__loggerFxn8__C                        
8000f390  ti_sysbios_family_c64p_Hwi_Module__loggerObj__C                         
8001322c  ti_sysbios_family_c64p_Hwi_Module__root__V                              
8000c080  ti_sysbios_family_c64p_Hwi_Module__startupDone__F                       
8000c080  ti_sysbios_family_c64p_Hwi_Module__startupDone__S                       
80013234  ti_sysbios_family_c64p_Hwi_Module__state__V                             
80007320  ti_sysbios_family_c64p_Hwi_Module_startup__E                            
800137b0  ti_sysbios_family_c64p_Hwi_Object__table__V                             
8000c0a0  ti_sysbios_family_c64p_Hwi_clearInterrupt__E                            
8000b680  ti_sysbios_family_c64p_Hwi_disableInterrupt__E                          
80005580  ti_sysbios_family_c64p_Hwi_dispatchAlways                               
80009940  ti_sysbios_family_c64p_Hwi_dispatchC__I                                 
80004820  ti_sysbios_family_c64p_Hwi_dispatchCore__I                              
8000b6c0  ti_sysbios_family_c64p_Hwi_enableInterrupt__E                           
800099e0  ti_sysbios_family_c64p_Hwi_getStackInfo__E                              
80013c00  ti_sysbios_family_c64p_Hwi_int0                                         
80013c20  ti_sysbios_family_c64p_Hwi_int1                                         
80013d40  ti_sysbios_family_c64p_Hwi_int10                                        
80013d60  ti_sysbios_family_c64p_Hwi_int11                                        
80013d80  ti_sysbios_family_c64p_Hwi_int12                                        
80013da0  ti_sysbios_family_c64p_Hwi_int13                                        
80013dc0  ti_sysbios_family_c64p_Hwi_int14                                        
80013de0  ti_sysbios_family_c64p_Hwi_int15                                        
80013c40  ti_sysbios_family_c64p_Hwi_int2                                         
80013c60  ti_sysbios_family_c64p_Hwi_int3                                         
80013c80  ti_sysbios_family_c64p_Hwi_int4                                         
80013ca0  ti_sysbios_family_c64p_Hwi_int5                                         
80013cc0  ti_sysbios_family_c64p_Hwi_int6                                         
80013ce0  ti_sysbios_family_c64p_Hwi_int7                                         
80013d00  ti_sysbios_family_c64p_Hwi_int8                                         
80013d20  ti_sysbios_family_c64p_Hwi_int9                                         
8000c0c0  ti_sysbios_family_c64p_Hwi_startup__E                                   
8000ace0  ti_sysbios_family_c64p_Hwi_switchAndDispatch__I                         
8000c0e0  ti_sysbios_family_c64p_Hwi_switchFromBootStack__E                       
8000c100  ti_sysbios_family_c64p_TimestampProvider_Module_startup__E              
8000c120  ti_sysbios_family_c64p_TimestampProvider_get32__E                       
8000c140  ti_sysbios_family_c64p_TimestampProvider_get64__E                       
8000bf80  ti_sysbios_family_c64p_TimestampProvider_getFreq__E                     
8000f394  ti_sysbios_family_c66_Cache_E_invalidL1CacheSize__C                     
8000f398  ti_sysbios_family_c66_Cache_E_invalidL2CacheSize__C                     
8000f594  ti_sysbios_family_c66_Cache_Module__id__C                               
8000af20  ti_sysbios_family_c66_Cache_Module_startup__E                           
8000c160  ti_sysbios_family_c66_Cache_RTSSynchInv__I                              
8000c180  ti_sysbios_family_c66_Cache_RTSSynchWbInv__I                            
8000c1a0  ti_sysbios_family_c66_Cache_RTSSynchWb__I                               
8000f39c  ti_sysbios_family_c66_Cache_atomicBlockSize__C                          
80006920  ti_sysbios_family_c66_Cache_block__I                                    
80007460  ti_sysbios_family_c66_Cache_getL1DInitSize__I                           
800075a0  ti_sysbios_family_c66_Cache_getL1PInitSize__I                           
80006460  ti_sysbios_family_c66_Cache_getL2InitSize__I                            
00008000  ti_sysbios_family_c66_Cache_l1dSize                                     
00008000  ti_sysbios_family_c66_Cache_l1pSize                                     
00000000  ti_sysbios_family_c66_Cache_l2Size                                      
8000ea00  ti_sysbios_family_c66_Cache_marvalues__C                                
8000f596  ti_sysbios_family_c66_Cache_registerRTSSynch__C                         
800076e0  ti_sysbios_family_c66_Cache_startup__I                                  
8000c1c0  ti_sysbios_family_c66_Cache_wait__E                                     
8000c1e0  ti_sysbios_family_shared_vayu_TimerSupport_Module__startupDone__F       
8000c1e0  ti_sysbios_family_shared_vayu_TimerSupport_Module__startupDone__S       
8000c200  ti_sysbios_family_shared_vayu_TimerSupport_Module_startup__E            
8000c220  ti_sysbios_family_shared_vayu_TimerSupport_enable__E                    
8000ad40  ti_sysbios_family_xxx_Hwi_switchAndRunFunc                              
8000b700  ti_sysbios_gates_GateHwi_Handle__label__S                               
8000c240  ti_sysbios_gates_GateHwi_Instance_init__E                               
8000f150  ti_sysbios_gates_GateHwi_Module__FXNS__C                                
800132a0  ti_sysbios_gates_GateHwi_Module__root__V                                
8000f1e0  ti_sysbios_gates_GateHwi_Object__DESC__C                                
8000f2dc  ti_sysbios_gates_GateHwi_Object__PARAMS__C                              
8000a280  ti_sysbios_gates_GateHwi_Object__create__S                              
8000b740  ti_sysbios_gates_GateHwi_Object__delete__S                              
80013808  ti_sysbios_gates_GateHwi_Object__table__V                               
8000c260  ti_sysbios_gates_GateHwi_enter__E                                       
8000c280  ti_sysbios_gates_GateHwi_leave__E                                       
8000c2a0  ti_sysbios_gates_GateHwi_query__E                                       
8000f3a0  ti_sysbios_gates_GateMutex_A_badContext__C                              
8000b780  ti_sysbios_gates_GateMutex_Handle__label__S                             
8000f3a4  ti_sysbios_gates_GateMutex_Instance_State_sem__O                        
8000c2c0  ti_sysbios_gates_GateMutex_Instance_finalize__E                         
8000b7c0  ti_sysbios_gates_GateMutex_Instance_init__E                             
8000f174  ti_sysbios_gates_GateMutex_Module__FXNS__C                              
8000f3a8  ti_sysbios_gates_GateMutex_Module__diagsEnabled__C                      
8000f3ac  ti_sysbios_gates_GateMutex_Module__diagsIncluded__C                     
8000f3b0  ti_sysbios_gates_GateMutex_Module__diagsMask__C                         
8000f598  ti_sysbios_gates_GateMutex_Module__id__C                                
800132a8  ti_sysbios_gates_GateMutex_Module__root__V                              
8000f200  ti_sysbios_gates_GateMutex_Object__DESC__C                              
8000f2f4  ti_sysbios_gates_GateMutex_Object__PARAMS__C                            
8000a300  ti_sysbios_gates_GateMutex_Object__create__S                            
8000af80  ti_sysbios_gates_GateMutex_Object__delete__S                            
800136d8  ti_sysbios_gates_GateMutex_Object__table__V                             
80005780  ti_sysbios_gates_GateMutex_enter__E                                     
8000b800  ti_sysbios_gates_GateMutex_leave__E                                     
8000c2e0  ti_sysbios_gates_GateMutex_query__E                                     
8000f3b4  ti_sysbios_hal_Hwi_E_stackOverflow__C                                   
8000c080  ti_sysbios_hal_Hwi_HwiProxy_Module__startupDone__S                      
8000c0a0  ti_sysbios_hal_Hwi_HwiProxy_clearInterrupt__E                           
8000b680  ti_sysbios_hal_Hwi_HwiProxy_disableInterrupt__E                         
8000b6c0  ti_sysbios_hal_Hwi_HwiProxy_enableInterrupt__E                          
800099e0  ti_sysbios_hal_Hwi_HwiProxy_getStackInfo__E                             
8000c0c0  ti_sysbios_hal_Hwi_HwiProxy_startup__E                                  
8000c0e0  ti_sysbios_hal_Hwi_HwiProxy_switchFromBootStack__E                      
8000f59a  ti_sysbios_hal_Hwi_Module__id__C                                        
800132b0  ti_sysbios_hal_Hwi_Module__root__V                                      
8000c300  ti_sysbios_hal_Hwi_Module_startup__E                                    
80013800  ti_sysbios_hal_Hwi_Object__table__V                                     
8000a380  ti_sysbios_hal_Hwi_checkStack                                           
8000a400  ti_sysbios_hal_Hwi_initStack                                            
8000f3b8  ti_sysbios_heaps_HeapMem_A_align__C                                     
8000f3bc  ti_sysbios_heaps_HeapMem_A_heapSize__C                                  
8000f3c0  ti_sysbios_heaps_HeapMem_A_invalidFree__C                               
8000f3c4  ti_sysbios_heaps_HeapMem_A_zeroBlock__C                                 
8000f3c8  ti_sysbios_heaps_HeapMem_E_memory__C                                    
8000b840  ti_sysbios_heaps_HeapMem_Handle__label__S                               
800115d0  ti_sysbios_heaps_HeapMem_Instance_State_0_buf__A                        
80003b00  ti_sysbios_heaps_HeapMem_Instance_init__E                               
8000b780  ti_sysbios_heaps_HeapMem_Module_GateProxy_Handle__label__S              
8000af80  ti_sysbios_heaps_HeapMem_Module_GateProxy_Object__delete__S             
8000c320  ti_sysbios_heaps_HeapMem_Module_GateProxy_enter__E                      
8000c340  ti_sysbios_heaps_HeapMem_Module_GateProxy_leave__E                      
8000c2e0  ti_sysbios_heaps_HeapMem_Module_GateProxy_query__E                      
8000f100  ti_sysbios_heaps_HeapMem_Module__FXNS__C                                
8000f3cc  ti_sysbios_heaps_HeapMem_Module__diagsEnabled__C                        
8000f3d0  ti_sysbios_heaps_HeapMem_Module__diagsIncluded__C                       
8000f3d4  ti_sysbios_heaps_HeapMem_Module__diagsMask__C                           
8000f3d8  ti_sysbios_heaps_HeapMem_Module__gateObj__C                             
8000f59c  ti_sysbios_heaps_HeapMem_Module__id__C                                  
800132b8  ti_sysbios_heaps_HeapMem_Module__root__V                                
8000f220  ti_sysbios_heaps_HeapMem_Object__DESC__C                                
8000f198  ti_sysbios_heaps_HeapMem_Object__PARAMS__C                              
8000f3dc  ti_sysbios_heaps_HeapMem_Object__count__C                               
8000a480  ti_sysbios_heaps_HeapMem_Object__create__S                              
8000b880  ti_sysbios_heaps_HeapMem_Object__delete__S                              
8000b8c0  ti_sysbios_heaps_HeapMem_Object__get__S                                 
800137c8  ti_sysbios_heaps_HeapMem_Object__table__V                               
800017e0  ti_sysbios_heaps_HeapMem_allocUnprotected__E                            
800090c0  ti_sysbios_heaps_HeapMem_alloc__E                                       
80001e20  ti_sysbios_heaps_HeapMem_freeUnprotected__E                             
8000afe0  ti_sysbios_heaps_HeapMem_free__E                                        
80009180  ti_sysbios_heaps_HeapMem_getStats__E                                    
80009a80  ti_sysbios_heaps_HeapMem_init__I                                        
8000c360  ti_sysbios_heaps_HeapMem_isBlocking__E                                  
8000f3e0  ti_sysbios_heaps_HeapMem_reqAlign__C                                    
8000f3e4  ti_sysbios_knl_Clock_LM_begin__C                                        
8000f3e8  ti_sysbios_knl_Clock_LM_tick__C                                         
8000f3ec  ti_sysbios_knl_Clock_LW_delayed__C                                      
8000f3f0  ti_sysbios_knl_Clock_Module_State_clockQ__O                             
8000f3f4  ti_sysbios_knl_Clock_Module__diagsEnabled__C                            
8000f3f8  ti_sysbios_knl_Clock_Module__diagsIncluded__C                           
8000f3fc  ti_sysbios_knl_Clock_Module__diagsMask__C                               
8000f59e  ti_sysbios_knl_Clock_Module__id__C                                      
8000f5a0  ti_sysbios_knl_Clock_Module__loggerDefined__C                           
8000f400  ti_sysbios_knl_Clock_Module__loggerFxn1__C                              
8000f404  ti_sysbios_knl_Clock_Module__loggerFxn2__C                              
8000f408  ti_sysbios_knl_Clock_Module__loggerObj__C                               
800132c0  ti_sysbios_knl_Clock_Module__root__V                                    
800132c8  ti_sysbios_knl_Clock_Module__state__V                                   
8000b040  ti_sysbios_knl_Clock_Module_startup__E                                  
8000c500  ti_sysbios_knl_Clock_TimerProxy_Module__startupDone__S                  
8000c380  ti_sysbios_knl_Clock_TimerProxy_getMaxTicks__E                          
80008b00  ti_sysbios_knl_Clock_TimerProxy_startup__E                              
8000a500  ti_sysbios_knl_Clock_doTick__I                                          
80009240  ti_sysbios_knl_Clock_logTick__E                                         
80003de0  ti_sysbios_knl_Clock_workFunc__E                                        
8000f410  ti_sysbios_knl_Idle_funcList__A                                         
8000f344  ti_sysbios_knl_Idle_funcList__C                                         
8000c3a0  ti_sysbios_knl_Idle_loop__E                                             
8000a580  ti_sysbios_knl_Idle_run__E                                              
8000c3c0  ti_sysbios_knl_Queue_Instance_init__E                                   
800132f4  ti_sysbios_knl_Queue_Module__root__V                                    
8000f240  ti_sysbios_knl_Queue_Object__DESC__C                                    
8000f30c  ti_sysbios_knl_Queue_Object__PARAMS__C                                  
8000c3e0  ti_sysbios_knl_Queue_Object__destruct__S                                
8000c400  ti_sysbios_knl_Queue_Object__get__S                                     
8000b0a0  ti_sysbios_knl_Queue_construct                                          
8000c420  ti_sysbios_knl_Queue_destruct                                           
8000c440  ti_sysbios_knl_Queue_empty__E                                           
8000f40c  ti_sysbios_knl_Semaphore_A_badContext__C                                
8000f414  ti_sysbios_knl_Semaphore_A_noEvents__C                                  
8000f418  ti_sysbios_knl_Semaphore_A_overflow__C                                  
8000f41c  ti_sysbios_knl_Semaphore_A_pendTaskDisabled__C                          
8000f420  ti_sysbios_knl_Semaphore_Instance_State_pendQ__O                        
8000c460  ti_sysbios_knl_Semaphore_Instance_finalize__E                           
80007820  ti_sysbios_knl_Semaphore_Instance_init__E                               
8000f424  ti_sysbios_knl_Semaphore_LM_pend__C                                     
8000f428  ti_sysbios_knl_Semaphore_LM_post__C                                     
8000f42c  ti_sysbios_knl_Semaphore_Module__diagsEnabled__C                        
8000f430  ti_sysbios_knl_Semaphore_Module__diagsIncluded__C                       
8000f434  ti_sysbios_knl_Semaphore_Module__diagsMask__C                           
8000f5a2  ti_sysbios_knl_Semaphore_Module__id__C                                  
8000f5a4  ti_sysbios_knl_Semaphore_Module__loggerDefined__C                       
8000f438  ti_sysbios_knl_Semaphore_Module__loggerFxn2__C                          
8000f43c  ti_sysbios_knl_Semaphore_Module__loggerFxn4__C                          
8000f440  ti_sysbios_knl_Semaphore_Module__loggerObj__C                           
800132fc  ti_sysbios_knl_Semaphore_Module__root__V                                
8000f260  ti_sysbios_knl_Semaphore_Object__DESC__C                                
8000f1bc  ti_sysbios_knl_Semaphore_Object__PARAMS__C                              
8000b900  ti_sysbios_knl_Semaphore_Object__destruct__S                            
8000b100  ti_sysbios_knl_Semaphore_construct                                      
8000c480  ti_sysbios_knl_Semaphore_destruct                                       
8000a600  ti_sysbios_knl_Semaphore_pendTimeout__I                                 
80000880  ti_sysbios_knl_Semaphore_pend__E                                        
80004080  ti_sysbios_knl_Semaphore_post__E                                        
8000f444  ti_sysbios_knl_Swi_LD_end__C                                            
8000f448  ti_sysbios_knl_Swi_LM_begin__C                                          
8000f44c  ti_sysbios_knl_Swi_LM_post__C                                           
800134a8  ti_sysbios_knl_Swi_Module_State_0_readyQ__A                             
8000f450  ti_sysbios_knl_Swi_Module__diagsEnabled__C                              
8000f454  ti_sysbios_knl_Swi_Module__diagsIncluded__C                             
8000f458  ti_sysbios_knl_Swi_Module__diagsMask__C                                 
8000f5a6  ti_sysbios_knl_Swi_Module__id__C                                        
8000f5a8  ti_sysbios_knl_Swi_Module__loggerDefined__C                             
8000f45c  ti_sysbios_knl_Swi_Module__loggerFxn1__C                                
8000f460  ti_sysbios_knl_Swi_Module__loggerFxn4__C                                
8000f464  ti_sysbios_knl_Swi_Module__loggerObj__C                                 
80013304  ti_sysbios_knl_Swi_Module__root__V                                      
8001330c  ti_sysbios_knl_Swi_Module__state__V                                     
8000b160  ti_sysbios_knl_Swi_Module_startup__E                                    
8000f468  ti_sysbios_knl_Swi_Object__count__C                                     
8000b940  ti_sysbios_knl_Swi_Object__get__S                                       
80013758  ti_sysbios_knl_Swi_Object__table__V                                     
8000c4a0  ti_sysbios_knl_Swi_disable__E                                           
80006f20  ti_sysbios_knl_Swi_post__E                                              
80007aa0  ti_sysbios_knl_Swi_restoreHwi__E                                        
80008940  ti_sysbios_knl_Swi_runLoop__I                                           
80005140  ti_sysbios_knl_Swi_run__I                                               
80008380  ti_sysbios_knl_Swi_schedule__I                                          
80008a20  ti_sysbios_knl_Swi_startup__E                                           
8000f46c  ti_sysbios_knl_Task_A_badPriority__C                                    
8000f470  ti_sysbios_knl_Task_A_badTaskState__C                                   
8000f474  ti_sysbios_knl_Task_A_badThreadType__C                                  
8000f478  ti_sysbios_knl_Task_A_badTimeout__C                                     
8000f47c  ti_sysbios_knl_Task_A_noPendElem__C                                     
8000f480  ti_sysbios_knl_Task_A_sleepTaskDisabled__C                              
8000f484  ti_sysbios_knl_Task_E_spOutOfBounds__C                                  
8000f488  ti_sysbios_knl_Task_E_stackOverflow__C                                  
800125d0  ti_sysbios_knl_Task_Instance_State_0_stack__A                           
800023e0  ti_sysbios_knl_Task_Instance_finalize__E                                
800030e0  ti_sysbios_knl_Task_Instance_init__E                                    
8000f48c  ti_sysbios_knl_Task_LD_block__C                                         
8000f490  ti_sysbios_knl_Task_LD_exit__C                                          
8000f494  ti_sysbios_knl_Task_LD_ready__C                                         
8000f498  ti_sysbios_knl_Task_LM_sleep__C                                         
8000f49c  ti_sysbios_knl_Task_LM_switch__C                                        
80013810  ti_sysbios_knl_Task_Module_State_0_idleTask__A                          
80013528  ti_sysbios_knl_Task_Module_State_0_readyQ__A                            
8000f4a0  ti_sysbios_knl_Task_Module_State_inactiveQ__O                           
8000f4a4  ti_sysbios_knl_Task_Module__diagsEnabled__C                             
8000f4a8  ti_sysbios_knl_Task_Module__diagsIncluded__C                            
8000f4ac  ti_sysbios_knl_Task_Module__diagsMask__C                                
8000f5aa  ti_sysbios_knl_Task_Module__id__C                                       
8000f5ac  ti_sysbios_knl_Task_Module__loggerDefined__C                            
8000f4b0  ti_sysbios_knl_Task_Module__loggerFxn2__C                               
8000f4b4  ti_sysbios_knl_Task_Module__loggerFxn4__C                               
8000f4b8  ti_sysbios_knl_Task_Module__loggerObj__C                                
80013328  ti_sysbios_knl_Task_Module__root__V                                     
80013330  ti_sysbios_knl_Task_Module__state__V                                    
80003800  ti_sysbios_knl_Task_Module_startup__E                                   
8000f280  ti_sysbios_knl_Task_Object__DESC__C                                     
8000f024  ti_sysbios_knl_Task_Object__PARAMS__C                                   
8000f4bc  ti_sysbios_knl_Task_Object__count__C                                    
8000b980  ti_sysbios_knl_Task_Object__get__S                                      
80013688  ti_sysbios_knl_Task_Object__table__V                                    
8000c020  ti_sysbios_knl_Task_SupportProxy_Module__startupDone__S                 
8000c040  ti_sysbios_knl_Task_SupportProxy_checkStack__E                          
8000c060  ti_sysbios_knl_Task_SupportProxy_getStackAlignment__E                   
8000aec0  ti_sysbios_knl_Task_SupportProxy_start__E                               
8000a100  ti_sysbios_knl_Task_SupportProxy_swap__E                                
8000f4c0  ti_sysbios_knl_Task_allBlockedFunc__C                                   
80009300  ti_sysbios_knl_Task_allBlockedFunction__I                               
80007960  ti_sysbios_knl_Task_blockI__E                                           
80005960  ti_sysbios_knl_Task_checkStacks__E                                      
800093c0  ti_sysbios_knl_Task_create                                              
8000f4c4  ti_sysbios_knl_Task_defaultStackHeap__C                                 
8000f4c8  ti_sysbios_knl_Task_defaultStackSize__C                                 
8000c4c0  ti_sysbios_knl_Task_disable__E                                          
8000b1c0  ti_sysbios_knl_Task_enter__I                                            
80005b40  ti_sysbios_knl_Task_exit__E                                             
8000f4cc  ti_sysbios_knl_Task_numConstructedTasks__C                              
80007080  ti_sysbios_knl_Task_postInit__I                                         
8000a680  ti_sysbios_knl_Task_processVitalTaskFlag__I                             
8000a700  ti_sysbios_knl_Task_restore__E                                          
80006600  ti_sysbios_knl_Task_schedule__I                                         
8000b9c0  ti_sysbios_knl_Task_sleepTimeout__I                                     
800028a0  ti_sysbios_knl_Task_sleep__E                                            
80006aa0  ti_sysbios_knl_Task_startCore__E                                        
8000c4e0  ti_sysbios_knl_Task_startup__E                                          
80008480  ti_sysbios_knl_Task_unblockI__E                                         
80013374  ti_sysbios_rts_ti_ThreadLocalStorage_Module__state__V                   
8000f4d0  ti_sysbios_timers_dmtimer_Timer_E_cannotSupport__C                      
8000f4d4  ti_sysbios_timers_dmtimer_Timer_E_freqMismatch__C                       
800133e8  ti_sysbios_timers_dmtimer_Timer_Module_State_0_device__A                
80013718  ti_sysbios_timers_dmtimer_Timer_Module_State_0_handles__A               
800135a8  ti_sysbios_timers_dmtimer_Timer_Module_State_0_intFreqs__A              
8000f4d8  ti_sysbios_timers_dmtimer_Timer_Module__diagsEnabled__C                 
8000f4dc  ti_sysbios_timers_dmtimer_Timer_Module__diagsIncluded__C                
8000f4e0  ti_sysbios_timers_dmtimer_Timer_Module__diagsMask__C                    
8000f5ae  ti_sysbios_timers_dmtimer_Timer_Module__id__C                           
80013380  ti_sysbios_timers_dmtimer_Timer_Module__root__V                         
8000c500  ti_sysbios_timers_dmtimer_Timer_Module__startupDone__F                  
8000c500  ti_sysbios_timers_dmtimer_Timer_Module__startupDone__S                  
80013388  ti_sysbios_timers_dmtimer_Timer_Module__state__V                        
80007bc0  ti_sysbios_timers_dmtimer_Timer_Module_startup__E                       
80013628  ti_sysbios_timers_dmtimer_Timer_Object__table__V                        
8000c1e0  ti_sysbios_timers_dmtimer_Timer_TimerSupportProxy_Module__startupDone__S
8000c220  ti_sysbios_timers_dmtimer_Timer_TimerSupportProxy_enable__E             
80002d20  ti_sysbios_timers_dmtimer_Timer_checkFreq__I                            
8000f5b0  ti_sysbios_timers_dmtimer_Timer_checkFrequency__C                       
80003480  ti_sysbios_timers_dmtimer_Timer_deviceConfig__I                         
8000c520  ti_sysbios_timers_dmtimer_Timer_getMaxTicks__E                          
80007ce0  ti_sysbios_timers_dmtimer_Timer_initDevice__I                           
8000f4e4  ti_sysbios_timers_dmtimer_Timer_numTimerDevices__C                      
80004320  ti_sysbios_timers_dmtimer_Timer_setPeriodMicroSecs__E                   
80006c20  ti_sysbios_timers_dmtimer_Timer_start__E                                
8000f5b2  ti_sysbios_timers_dmtimer_Timer_startupNeeded__C                        
80008b00  ti_sysbios_timers_dmtimer_Timer_startup__E                              
80009480  ti_sysbios_timers_dmtimer_Timer_stop__E                                 
8000ba00  ti_sysbios_timers_dmtimer_Timer_stub__E                                 
8000f4e8  xdc_runtime_Assert_E_assertFailed__C                                    
80009b20  xdc_runtime_Assert_raise__I                                             
8000f4ec  xdc_runtime_Core_A_initializedParams__C                                 
8000f4f0  xdc_runtime_Core_Module__diagsEnabled__C                                
8000f4f4  xdc_runtime_Core_Module__diagsIncluded__C                               
8000f4f8  xdc_runtime_Core_Module__diagsMask__C                                   
8000f5b4  xdc_runtime_Core_Module__id__C                                          
8000a780  xdc_runtime_Core_assignLabel__I                                         
8000a800  xdc_runtime_Core_assignParams__I                                        
80006da0  xdc_runtime_Core_constructObject__I                                     
80005360  xdc_runtime_Core_createObject__I                                        
80007e00  xdc_runtime_Core_deleteObject__I                                        
8000f4fc  xdc_runtime_Error_E_memory__C                                           
8000f500  xdc_runtime_Error_Module__diagsEnabled__C                               
8000f504  xdc_runtime_Error_Module__diagsIncluded__C                              
8000f508  xdc_runtime_Error_Module__diagsMask__C                                  
8000f5b6  xdc_runtime_Error_Module__loggerDefined__C                              
8000f50c  xdc_runtime_Error_Module__loggerFxn8__C                                 
8000f510  xdc_runtime_Error_Module__loggerObj__C                                  
8001339c  xdc_runtime_Error_Module__state__V                                      
8000ba40  xdc_runtime_Error_check__E                                              
8000c540  xdc_runtime_Error_getSite__E                                            
8000ba80  xdc_runtime_Error_init__E                                               
8000f5b8  xdc_runtime_Error_maxDepth__C                                           
80005d20  xdc_runtime_Error_policyDefault__E                                      
8000f514  xdc_runtime_Error_policyFxn__C                                          
8000f518  xdc_runtime_Error_policy__C                                             
80008be0  xdc_runtime_Error_print__E                                              
8000f51c  xdc_runtime_Error_raiseHook__C                                          
8000c560  xdc_runtime_Error_raiseX__E                                             
80009bc0  xdc_runtime_Error_setX__E                                               
8000c580  xdc_runtime_Gate_enterSystem__E                                         
8000c5a0  xdc_runtime_Gate_leaveSystem__E                                         
8000f520  xdc_runtime_IFilterLogger_Interface__BASE__C                            
8000f524  xdc_runtime_IGateProvider_Interface__BASE__C                            
8000f528  xdc_runtime_IHeap_Interface__BASE__C                                    
8000f52c  xdc_runtime_ILogger_Interface__BASE__C                                  
8000f530  xdc_runtime_IModule_Interface__BASE__C                                  
8000f534  xdc_runtime_Log_L_error__C                                              
8000f538  xdc_runtime_LoggerBuf_E_badLevel__C                                     
8000bac0  xdc_runtime_LoggerBuf_Handle__label__S                                  
80012dd0  xdc_runtime_LoggerBuf_Instance_State_0_entryArr__A                      
8000bb00  xdc_runtime_LoggerBuf_Instance_finalize__E                              
8000a880  xdc_runtime_LoggerBuf_Instance_init__E                                  
8000b700  xdc_runtime_LoggerBuf_Module_GateProxy_Handle__label__S                 
8000b740  xdc_runtime_LoggerBuf_Module_GateProxy_Object__delete__S                
8000c600  xdc_runtime_LoggerBuf_Module_GateProxy_enter__E                         
8000c620  xdc_runtime_LoggerBuf_Module_GateProxy_leave__E                         
8000c2a0  xdc_runtime_LoggerBuf_Module_GateProxy_query__E                         
8000f060  xdc_runtime_LoggerBuf_Module__FXNS__C                                   
8000f53c  xdc_runtime_LoggerBuf_Module__gateObj__C                                
8000f5ba  xdc_runtime_LoggerBuf_Module__id__C                                     
800133a0  xdc_runtime_LoggerBuf_Module__root__V                                   
800133a8  xdc_runtime_LoggerBuf_Module__state__V                                  
8000a900  xdc_runtime_LoggerBuf_Module_startup__E                                 
8000f2a0  xdc_runtime_LoggerBuf_Object__DESC__C                                   
8000f128  xdc_runtime_LoggerBuf_Object__PARAMS__C                                 
8000f540  xdc_runtime_LoggerBuf_Object__count__C                                  
80009c60  xdc_runtime_LoggerBuf_Object__create__S                                 
8000b220  xdc_runtime_LoggerBuf_Object__delete__S                                 
8000bb40  xdc_runtime_LoggerBuf_Object__get__S                                    
80013788  xdc_runtime_LoggerBuf_Object__table__V                                  
8000c120  xdc_runtime_LoggerBuf_TimestampProxy_get32__E                           
8000c140  xdc_runtime_LoggerBuf_TimestampProxy_get64__E                           
8000bf80  xdc_runtime_LoggerBuf_TimestampProxy_getFreq__E                         
8000c640  xdc_runtime_LoggerBuf_disable__E                                        
8000c660  xdc_runtime_LoggerBuf_enable__E                                         
8000f5bc  xdc_runtime_LoggerBuf_filterByLevel__C                                  
8000a980  xdc_runtime_LoggerBuf_filterOutEvent__I                                 
80008580  xdc_runtime_LoggerBuf_getFilterLevel__E                                 
8000bb80  xdc_runtime_LoggerBuf_reset__E                                          
80007f20  xdc_runtime_LoggerBuf_setFilterLevel__E                                 
8000f544  xdc_runtime_LoggerBuf_statusLogger__C                                   
8000bbc0  xdc_runtime_LoggerBuf_write0__E                                         
8000c680  xdc_runtime_LoggerBuf_write1__E                                         
8000c6a0  xdc_runtime_LoggerBuf_write2__E                                         
800060e0  xdc_runtime_LoggerBuf_write4__E                                         
800045a0  xdc_runtime_LoggerBuf_write8__E                                         
8000b700  xdc_runtime_Main_Module_GateProxy_Handle__label__S                      
8000b740  xdc_runtime_Main_Module_GateProxy_Object__delete__S                     
8000c2a0  xdc_runtime_Main_Module_GateProxy_query__E                              
8000b840  xdc_runtime_Memory_HeapProxy_Handle__label__S                           
8000b880  xdc_runtime_Memory_HeapProxy_Object__delete__S                          
8000c5c0  xdc_runtime_Memory_HeapProxy_alloc__E                                   
8000c5e0  xdc_runtime_Memory_HeapProxy_free__E                                    
8000f5be  xdc_runtime_Memory_Module__id__C                                        
800133b0  xdc_runtime_Memory_Module__state__V                                     
80008cc0  xdc_runtime_Memory_alloc__E                                             
8000c6c0  xdc_runtime_Memory_calloc__E                                            
8000f548  xdc_runtime_Memory_defaultHeapInstance__C                               
8000bc00  xdc_runtime_Memory_free__E                                              
8000c6e0  xdc_runtime_Memory_getMaxDefaultTypeAlign__E                            
8000b280  xdc_runtime_Memory_valloc__E                                            
800133b4  xdc_runtime_Registry_Module__state__V                                   
8000bc40  xdc_runtime_Registry_findById__E                                        
800133bc  xdc_runtime_Startup_Module__state__V                                    
00000001  xdc_runtime_Startup__EXECFXN__C                                         
00000001  xdc_runtime_Startup__RESETFXN__C                                        
8000f54c  xdc_runtime_Startup_execImpl__C                                         
80008680  xdc_runtime_Startup_exec__E                                             
8000c700  xdc_runtime_Startup_exec__I                                             
8000f350  xdc_runtime_Startup_firstFxns__A                                        
8000f358  xdc_runtime_Startup_firstFxns__C                                        
8000f360  xdc_runtime_Startup_lastFxns__C                                         
8000f550  xdc_runtime_Startup_maxPasses__C                                        
800076e0  xdc_runtime_Startup_reset__I                                            
8000c720  xdc_runtime_Startup_rtsDone__E                                          
8000f2c0  xdc_runtime_Startup_sfxnRts__A                                          
8000f554  xdc_runtime_Startup_sfxnRts__C                                          
8000f0a0  xdc_runtime_Startup_sfxnTab__A                                          
8000f558  xdc_runtime_Startup_sfxnTab__C                                          
80005f00  xdc_runtime_Startup_startMods__I                                        
80012fd0  xdc_runtime_SysMin_Module_State_0_outbuf__A                             
800133c4  xdc_runtime_SysMin_Module__state__V                                     
8000b2e0  xdc_runtime_SysMin_Module_startup__E                                    
80009d00  xdc_runtime_SysMin_abort__E                                             
8000f55c  xdc_runtime_SysMin_bufSize__C                                           
8000b340  xdc_runtime_SysMin_exit__E                                              
8000f5c0  xdc_runtime_SysMin_flushAtExit__C                                       
80009da0  xdc_runtime_SysMin_flush__E                                             
8000f560  xdc_runtime_SysMin_outputFunc__C                                        
8000aa00  xdc_runtime_SysMin_output__I                                            
80009e40  xdc_runtime_SysMin_putch__E                                             
8000c740  xdc_runtime_SysMin_ready__E                                             
8000b700  xdc_runtime_System_Module_GateProxy_Handle__label__S                    
8000b740  xdc_runtime_System_Module_GateProxy_Object__delete__S                   
8000c760  xdc_runtime_System_Module_GateProxy_enter__E                            
8000c780  xdc_runtime_System_Module_GateProxy_leave__E                            
8000c2a0  xdc_runtime_System_Module_GateProxy_query__E                            
800137e0  xdc_runtime_System_Module_State_0_atexitHandlers__A                     
8000f564  xdc_runtime_System_Module__gateObj__C                                   
800133d0  xdc_runtime_System_Module__state__V                                     
8000c7a0  xdc_runtime_System_Module_startup__E                                    
80009d00  xdc_runtime_System_SupportProxy_abort__E                                
8000b340  xdc_runtime_System_SupportProxy_exit__E                                 
80009da0  xdc_runtime_System_SupportProxy_flush__E                                
80009e40  xdc_runtime_System_SupportProxy_putch__E                                
8000c740  xdc_runtime_System_SupportProxy_ready__E                                
8000f568  xdc_runtime_System_abortFxn__C                                          
8000bea0  xdc_runtime_System_abortStd__E                                          
8000bc80  xdc_runtime_System_abort__E                                             
8000bcc0  xdc_runtime_System_aprintf__E                                           
8000c7c0  xdc_runtime_System_aprintf_va__E                                        
8000c7c0  xdc_runtime_System_aprintf_va__F                                        
8000aa80  xdc_runtime_System_atexit__E                                            
8000b3a0  xdc_runtime_System_avprintf__E                                          
80000000  xdc_runtime_System_doPrint__I                                           
8000f56c  xdc_runtime_System_exitFxn__C                                           
80008f40  xdc_runtime_System_exitStd__E                                           
8000bd00  xdc_runtime_System_exit__E                                              
8000f570  xdc_runtime_System_extendFxn__C                                         
80009600  xdc_runtime_System_formatNum__I                                         
8000f574  xdc_runtime_System_maxAtexitHandlers__C                                 
80004f00  xdc_runtime_System_printfExtend__I                                      
8000bd40  xdc_runtime_System_printf__E                                            
8000c7e0  xdc_runtime_System_printf_va__E                                         
8000c7e0  xdc_runtime_System_printf_va__F                                         
8000ab00  xdc_runtime_System_processAtExit__E                                     
8000ab80  xdc_runtime_System_putchar__I                                           
8000b400  xdc_runtime_System_vprintf__E                                           
8000c800  xdc_runtime_System_vsnprintf__E                                         
800133d8  xdc_runtime_Text_Module__state__V                                       
8000f5c2  xdc_runtime_Text_charCnt__C                                             
8000c840  xdc_runtime_Text_charTab__A                                             
8000f578  xdc_runtime_Text_charTab__C                                             
8000b460  xdc_runtime_Text_cordText__E                                            
8000f5c4  xdc_runtime_Text_isLoaded__C                                            
8000f57c  xdc_runtime_Text_nameEmpty__C                                           
8000f580  xdc_runtime_Text_nameStatic__C                                          
8000f584  xdc_runtime_Text_nameUnknown__C                                         
8000ee00  xdc_runtime_Text_nodeTab__A                                             
8000f588  xdc_runtime_Text_nodeTab__C                                             
8000ac00  xdc_runtime_Text_printVisFxn__I                                         
80008040  xdc_runtime_Text_putLab__E                                              
80008160  xdc_runtime_Text_putMod__E                                              
800062a0  xdc_runtime_Text_putSite__E                                             
8000f5c6  xdc_runtime_Text_registryModsLastId__C                                  
8000bd80  xdc_runtime_Text_ropeText__E                                            
8000f5c8  xdc_runtime_Text_unnamedModsLastId__C                                   
80008da0  xdc_runtime_Text_visitRope2__I                                          
8000f58c  xdc_runtime_Text_visitRopeFxn__C                                        
8000c820  xdc_runtime_Text_visitRope__I                                           
80009ee0  xdc_runtime_Text_xprintf__I                                             
8000c120  xdc_runtime_Timestamp_SupportProxy_get32__E                             
8000c140  xdc_runtime_Timestamp_SupportProxy_get64__E                             
8000bf80  xdc_runtime_Timestamp_SupportProxy_getFreq__E                           


GLOBAL SYMBOLS: SORTED BY Symbol Address 

address   name                                                                    
-------   ----                                                                    
00000000  __TI_STATIC_BASE                                                        
00000000  _argsize                                                                
00000000  ti_sysbios_family_c66_Cache_l2Size                                      
00000001  xdc_runtime_Startup__EXECFXN__C                                         
00000001  xdc_runtime_Startup__RESETFXN__C                                        
00002000  __TI_STACK_SIZE                                                         
00008000  ti_sysbios_family_c66_Cache_l1dSize                                     
00008000  ti_sysbios_family_c66_Cache_l1pSize                                     
80000000  __ASM__                                                                 
80000000  xdc_runtime_System_doPrint__I                                           
80000070  __ISA__                                                                 
80000088  __PLAT__                                                                
800000b0  __TARG__                                                                
800000d8  __TRDR__                                                                
80000880  ti_sysbios_knl_Semaphore_pend__E                                        
80001060  ti_sysbios_family_c64p_Exception_handler__I                             
800017e0  ti_sysbios_heaps_HeapMem_allocUnprotected__E                            
80001e20  ti_sysbios_heaps_HeapMem_freeUnprotected__E                             
800023e0  ti_sysbios_knl_Task_Instance_finalize__E                                
800028a0  ti_sysbios_knl_Task_sleep__E                                            
80002d20  ti_sysbios_timers_dmtimer_Timer_checkFreq__I                            
800030e0  ti_sysbios_knl_Task_Instance_init__E                                    
80003480  ti_sysbios_timers_dmtimer_Timer_deviceConfig__I                         
80003800  ti_sysbios_knl_Task_Module_startup__E                                   
80003b00  ti_sysbios_heaps_HeapMem_Instance_init__E                               
80003de0  ti_sysbios_knl_Clock_workFunc__E                                        
80004080  ti_sysbios_knl_Semaphore_post__E                                        
80004320  ti_sysbios_timers_dmtimer_Timer_setPeriodMicroSecs__E                   
800045a0  xdc_runtime_LoggerBuf_write8__E                                         
80004820  ti_sysbios_family_c64p_Hwi_dispatchCore__I                              
80004a80  __c6xabi_divull                                                         
80004cc0  ti_sysbios_family_c64p_Exception_internalHandler__I                     
80004f00  xdc_runtime_System_printfExtend__I                                      
80005140  ti_sysbios_knl_Swi_run__I                                               
80005360  xdc_runtime_Core_createObject__I                                        
80005580  ti_sysbios_family_c64p_Hwi_dispatchAlways                               
80005780  ti_sysbios_gates_GateMutex_enter__E                                     
80005960  ti_sysbios_knl_Task_checkStacks__E                                      
80005b40  ti_sysbios_knl_Task_exit__E                                             
80005d20  xdc_runtime_Error_policyDefault__E                                      
80005f00  xdc_runtime_Startup_startMods__I                                        
800060e0  xdc_runtime_LoggerBuf_write4__E                                         
800062a0  xdc_runtime_Text_putSite__E                                             
80006460  ti_sysbios_family_c66_Cache_getL2InitSize__I                            
80006600  ti_sysbios_knl_Task_schedule__I                                         
800067a0  ti_sysbios_family_c64p_Exception_dispatch__E                            
80006920  ti_sysbios_family_c66_Cache_block__I                                    
80006aa0  ti_sysbios_knl_Task_startCore__E                                        
80006c20  ti_sysbios_timers_dmtimer_Timer_start__E                                
80006da0  xdc_runtime_Core_constructObject__I                                     
80006f20  ti_sysbios_knl_Swi_post__E                                              
80007080  ti_sysbios_knl_Task_postInit__I                                         
800071e0  _auto_init_elf                                                          
80007320  ti_sysbios_family_c64p_Hwi_Module_startup__E                            
80007460  ti_sysbios_family_c66_Cache_getL1DInitSize__I                           
800075a0  ti_sysbios_family_c66_Cache_getL1PInitSize__I                           
800076e0  ti_sysbios_family_c66_Cache_startup__I                                  
800076e0  xdc_runtime_Startup_reset__I                                            
80007820  ti_sysbios_knl_Semaphore_Instance_init__E                               
80007960  ti_sysbios_knl_Task_blockI__E                                           
80007aa0  ti_sysbios_knl_Swi_restoreHwi__E                                        
80007bc0  ti_sysbios_timers_dmtimer_Timer_Module_startup__E                       
80007ce0  ti_sysbios_timers_dmtimer_Timer_initDevice__I                           
80007e00  xdc_runtime_Core_deleteObject__I                                        
80007f20  xdc_runtime_LoggerBuf_setFilterLevel__E                                 
80008040  xdc_runtime_Text_putLab__E                                              
80008160  xdc_runtime_Text_putMod__E                                              
80008380  ti_sysbios_knl_Swi_schedule__I                                          
80008480  ti_sysbios_knl_Task_unblockI__E                                         
80008580  xdc_runtime_LoggerBuf_getFilterLevel__E                                 
80008680  xdc_runtime_Startup_exec__E                                             
80008780  HOSTwrite                                                               
80008860  memset                                                                  
80008940  ti_sysbios_knl_Swi_runLoop__I                                           
80008a20  ti_sysbios_knl_Swi_startup__E                                           
80008b00  ti_sysbios_knl_Clock_TimerProxy_startup__E                              
80008b00  ti_sysbios_timers_dmtimer_Timer_startup__E                              
80008be0  xdc_runtime_Error_print__E                                              
80008cc0  xdc_runtime_Memory_alloc__E                                             
80008da0  xdc_runtime_Text_visitRope2__I                                          
80008e80  __c6xabi_divu                                                           
80008e80  __divu                                                                  
80008f40  exit                                                                    
80008f40  xdc_runtime_System_exitStd__E                                           
80009000  taskFxn                                                                 
80009044  main                                                                    
800090c0  ti_sysbios_heaps_HeapMem_alloc__E                                       
80009180  ti_sysbios_heaps_HeapMem_getStats__E                                    
80009240  ti_sysbios_knl_Clock_logTick__E                                         
80009300  ti_sysbios_knl_Task_allBlockedFunction__I                               
800093c0  ti_sysbios_knl_Task_create                                              
80009480  ti_sysbios_timers_dmtimer_Timer_stop__E                                 
80009540  __TI_tls_init                                                           
80009600  xdc_runtime_System_formatNum__I                                         
800096c0  __c6xabi_remu                                                           
800096c0  __remu                                                                  
80009760  _c_int00                                                                
80009800  memcpy                                                                  
800098a0  ti_sysbios_family_c64p_Exception_Module_startup__E                      
80009940  ti_sysbios_family_c64p_Hwi_dispatchC__I                                 
800099e0  ti_sysbios_family_c64p_Hwi_getStackInfo__E                              
800099e0  ti_sysbios_hal_Hwi_HwiProxy_getStackInfo__E                             
80009a80  ti_sysbios_heaps_HeapMem_init__I                                        
80009b20  xdc_runtime_Assert_raise__I                                             
80009bc0  xdc_runtime_Error_setX__E                                               
80009c60  xdc_runtime_LoggerBuf_Object__create__S                                 
80009d00  xdc_runtime_SysMin_abort__E                                             
80009d00  xdc_runtime_System_SupportProxy_abort__E                                
80009da0  xdc_runtime_SysMin_flush__E                                             
80009da0  xdc_runtime_System_SupportProxy_flush__E                                
80009e40  xdc_runtime_SysMin_putch__E                                             
80009e40  xdc_runtime_System_SupportProxy_putch__E                                
80009ee0  xdc_runtime_Text_xprintf__I                                             
80009f80  __TI_readmsg                                                            
8000a000  __TI_writemsg                                                           
8000a060  C$$IO$$                                                                 
8000a080  __c6xabi_llshl                                                          
8000a100  ti_sysbios_family_c62_TaskSupport_swap__E                               
8000a100  ti_sysbios_knl_Task_SupportProxy_swap__E                                
8000a180  ti_sysbios_BIOS_atExitFunc__I                                           
8000a200  ti_sysbios_BIOS_registerRTSLock__I                                      
8000a280  ti_sysbios_gates_GateHwi_Object__create__S                              
8000a300  ti_sysbios_gates_GateMutex_Object__create__S                            
8000a380  ti_sysbios_hal_Hwi_checkStack                                           
8000a400  ti_sysbios_hal_Hwi_initStack                                            
8000a480  ti_sysbios_heaps_HeapMem_Object__create__S                              
8000a500  ti_sysbios_knl_Clock_doTick__I                                          
8000a580  ti_sysbios_knl_Idle_run__E                                              
8000a600  ti_sysbios_knl_Semaphore_pendTimeout__I                                 
8000a680  ti_sysbios_knl_Task_processVitalTaskFlag__I                             
8000a700  ti_sysbios_knl_Task_restore__E                                          
8000a780  xdc_runtime_Core_assignLabel__I                                         
8000a800  xdc_runtime_Core_assignParams__I                                        
8000a880  xdc_runtime_LoggerBuf_Instance_init__E                                  
8000a900  xdc_runtime_LoggerBuf_Module_startup__E                                 
8000a980  xdc_runtime_LoggerBuf_filterOutEvent__I                                 
8000aa00  xdc_runtime_SysMin_output__I                                            
8000aa80  xdc_runtime_System_atexit__E                                            
8000ab00  xdc_runtime_System_processAtExit__E                                     
8000ab80  xdc_runtime_System_putchar__I                                           
8000ac00  xdc_runtime_Text_printVisFxn__I                                         
8000ac80  __c6xabi_llshru                                                         
8000ace0  ti_sysbios_family_c64p_Hwi_switchAndDispatch__I                         
8000ad40  ti_sysbios_family_xxx_Hwi_switchAndRunFunc                              
8000ada0  ti_sysbios_BIOS_errorRaiseHook__I                                       
8000ae00  ti_sysbios_BIOS_removeRTSLock__I                                        
8000ae60  ti_sysbios_BIOS_startFunc__I                                            
8000aec0  ti_sysbios_family_c62_TaskSupport_start__E                              
8000aec0  ti_sysbios_knl_Task_SupportProxy_start__E                               
8000af20  ti_sysbios_family_c66_Cache_Module_startup__E                           
8000af80  ti_sysbios_BIOS_RtsGateProxy_Object__delete__S                          
8000af80  ti_sysbios_gates_GateMutex_Object__delete__S                            
8000af80  ti_sysbios_heaps_HeapMem_Module_GateProxy_Object__delete__S             
8000afe0  ti_sysbios_heaps_HeapMem_free__E                                        
8000b040  ti_sysbios_knl_Clock_Module_startup__E                                  
8000b0a0  ti_sysbios_knl_Queue_construct                                          
8000b100  ti_sysbios_knl_Semaphore_construct                                      
8000b160  ti_sysbios_knl_Swi_Module_startup__E                                    
8000b1c0  ti_sysbios_knl_Task_enter__I                                            
8000b220  xdc_runtime_LoggerBuf_Object__delete__S                                 
8000b280  xdc_runtime_Memory_valloc__E                                            
8000b2e0  xdc_runtime_SysMin_Module_startup__E                                    
8000b340  xdc_runtime_SysMin_exit__E                                              
8000b340  xdc_runtime_System_SupportProxy_exit__E                                 
8000b3a0  xdc_runtime_System_avprintf__E                                          
8000b400  xdc_runtime_System_vprintf__E                                           
8000b460  xdc_runtime_Text_cordText__E                                            
8000b4c0  __c6xabi_strasgi_64plus                                                 
8000b4c0  __strasgi_64plus                                                        
8000b500  _args_main                                                              
8000b540  _subcull                                                                
8000b580  ti_sysbios_family_c62_TaskSupport_buildTaskStack                        
8000b5c0  ti_sysbios_BIOS_exitFunc__I                                             
8000b600  ti_sysbios_BIOS_rtsLock__I                                              
8000b640  ti_sysbios_BIOS_rtsUnlock__I                                            
8000b680  ti_sysbios_family_c64p_Hwi_disableInterrupt__E                          
8000b680  ti_sysbios_hal_Hwi_HwiProxy_disableInterrupt__E                         
8000b6c0  ti_sysbios_family_c64p_Hwi_enableInterrupt__E                           
8000b6c0  ti_sysbios_hal_Hwi_HwiProxy_enableInterrupt__E                          
8000b700  ti_sysbios_gates_GateHwi_Handle__label__S                               
8000b700  xdc_runtime_LoggerBuf_Module_GateProxy_Handle__label__S                 
8000b700  xdc_runtime_Main_Module_GateProxy_Handle__label__S                      
8000b700  xdc_runtime_System_Module_GateProxy_Handle__label__S                    
8000b740  ti_sysbios_gates_GateHwi_Object__delete__S                              
8000b740  xdc_runtime_LoggerBuf_Module_GateProxy_Object__delete__S                
8000b740  xdc_runtime_Main_Module_GateProxy_Object__delete__S                     
8000b740  xdc_runtime_System_Module_GateProxy_Object__delete__S                   
8000b780  ti_sysbios_BIOS_RtsGateProxy_Handle__label__S                           
8000b780  ti_sysbios_gates_GateMutex_Handle__label__S                             
8000b780  ti_sysbios_heaps_HeapMem_Module_GateProxy_Handle__label__S              
8000b7c0  ti_sysbios_gates_GateMutex_Instance_init__E                             
8000b800  ti_sysbios_gates_GateMutex_leave__E                                     
8000b840  ti_sysbios_heaps_HeapMem_Handle__label__S                               
8000b840  xdc_runtime_Memory_HeapProxy_Handle__label__S                           
8000b880  ti_sysbios_heaps_HeapMem_Object__delete__S                              
8000b880  xdc_runtime_Memory_HeapProxy_Object__delete__S                          
8000b8c0  ti_sysbios_heaps_HeapMem_Object__get__S                                 
8000b900  ti_sysbios_knl_Semaphore_Object__destruct__S                            
8000b940  ti_sysbios_knl_Swi_Object__get__S                                       
8000b980  ti_sysbios_knl_Task_Object__get__S                                      
8000b9c0  ti_sysbios_knl_Task_sleepTimeout__I                                     
8000ba00  ti_sysbios_timers_dmtimer_Timer_stub__E                                 
8000ba40  xdc_runtime_Error_check__E                                              
8000ba80  xdc_runtime_Error_init__E                                               
8000bac0  xdc_runtime_LoggerBuf_Handle__label__S                                  
8000bb00  xdc_runtime_LoggerBuf_Instance_finalize__E                              
8000bb40  xdc_runtime_LoggerBuf_Object__get__S                                    
8000bb80  xdc_runtime_LoggerBuf_reset__E                                          
8000bbc0  xdc_runtime_LoggerBuf_write0__E                                         
8000bc00  xdc_runtime_Memory_free__E                                              
8000bc40  xdc_runtime_Registry_findById__E                                        
8000bc80  xdc_runtime_System_abort__E                                             
8000bcc0  xdc_runtime_System_aprintf__E                                           
8000bd00  xdc_runtime_System_exit__E                                              
8000bd40  xdc_runtime_System_printf__E                                            
8000bd80  xdc_runtime_Text_ropeText__E                                            
8000bdc0  LoggerBuf_instanceStartup                                               
8000bde0  __xdc__init                                                             
8000be00  _nop                                                                    
8000be20  _register_lock                                                          
8000be40  _register_synch_api                                                     
8000be60  _register_unlock                                                        
8000be80  ti_sysbios_family_c62_TaskSupport_glue                                  
8000bea0  C$$EXIT                                                                 
8000bea0  abort                                                                   
8000bea0  xdc_runtime_System_abortStd__E                                          
8000bec0  __TI_zero_init                                                          
8000bee0  __TI_decompress_none                                                    
8000bf00  __TI_decompress_rle24                                                   
8000bf20  ti_sysbios_BIOS_RtsGateProxy_enter__E                                   
8000bf40  ti_sysbios_BIOS_RtsGateProxy_leave__E                                   
8000bf60  ti_sysbios_BIOS_exit__E                                                 
8000bf80  ti_sysbios_BIOS_getCpuFreq__E                                           
8000bf80  ti_sysbios_family_c64p_TimestampProvider_getFreq__E                     
8000bf80  xdc_runtime_LoggerBuf_TimestampProxy_getFreq__E                         
8000bf80  xdc_runtime_Timestamp_SupportProxy_getFreq__E                           
8000bfa0  ti_sysbios_BIOS_linkedWithIncorrectBootLibrary__E                       
8000bfc0  ti_sysbios_BIOS_nullFunc__I                                             
8000bfe0  ti_sysbios_BIOS_setThreadType__E                                        
8000c000  ti_sysbios_BIOS_start__E                                                
8000c020  ti_sysbios_family_c62_TaskSupport_Module__startupDone__S                
8000c020  ti_sysbios_knl_Task_SupportProxy_Module__startupDone__S                 
8000c040  ti_sysbios_family_c62_TaskSupport_checkStack__E                         
8000c040  ti_sysbios_knl_Task_SupportProxy_checkStack__E                          
8000c060  ti_sysbios_family_c62_TaskSupport_getStackAlignment__E                  
8000c060  ti_sysbios_knl_Task_SupportProxy_getStackAlignment__E                   
8000c080  ti_sysbios_family_c64p_Hwi_Module__startupDone__F                       
8000c080  ti_sysbios_family_c64p_Hwi_Module__startupDone__S                       
8000c080  ti_sysbios_hal_Hwi_HwiProxy_Module__startupDone__S                      
8000c0a0  ti_sysbios_family_c64p_Hwi_clearInterrupt__E                            
8000c0a0  ti_sysbios_hal_Hwi_HwiProxy_clearInterrupt__E                           
8000c0c0  ti_sysbios_family_c64p_Hwi_startup__E                                   
8000c0c0  ti_sysbios_hal_Hwi_HwiProxy_startup__E                                  
8000c0e0  ti_sysbios_family_c64p_Hwi_switchFromBootStack__E                       
8000c0e0  ti_sysbios_hal_Hwi_HwiProxy_switchFromBootStack__E                      
8000c100  ti_sysbios_family_c64p_TimestampProvider_Module_startup__E              
8000c120  ti_sysbios_family_c64p_TimestampProvider_get32__E                       
8000c120  xdc_runtime_LoggerBuf_TimestampProxy_get32__E                           
8000c120  xdc_runtime_Timestamp_SupportProxy_get32__E                             
8000c140  ti_sysbios_family_c64p_TimestampProvider_get64__E                       
8000c140  xdc_runtime_LoggerBuf_TimestampProxy_get64__E                           
8000c140  xdc_runtime_Timestamp_SupportProxy_get64__E                             
8000c160  ti_sysbios_family_c66_Cache_RTSSynchInv__I                              
8000c180  ti_sysbios_family_c66_Cache_RTSSynchWbInv__I                            
8000c1a0  ti_sysbios_family_c66_Cache_RTSSynchWb__I                               
8000c1c0  ti_sysbios_family_c66_Cache_wait__E                                     
8000c1e0  ti_sysbios_family_shared_vayu_TimerSupport_Module__startupDone__F       
8000c1e0  ti_sysbios_family_shared_vayu_TimerSupport_Module__startupDone__S       
8000c1e0  ti_sysbios_timers_dmtimer_Timer_TimerSupportProxy_Module__startupDone__S
8000c200  ti_sysbios_family_shared_vayu_TimerSupport_Module_startup__E            
8000c220  ti_sysbios_family_shared_vayu_TimerSupport_enable__E                    
8000c220  ti_sysbios_timers_dmtimer_Timer_TimerSupportProxy_enable__E             
8000c240  ti_sysbios_gates_GateHwi_Instance_init__E                               
8000c260  ti_sysbios_gates_GateHwi_enter__E                                       
8000c280  ti_sysbios_gates_GateHwi_leave__E                                       
8000c2a0  ti_sysbios_gates_GateHwi_query__E                                       
8000c2a0  xdc_runtime_LoggerBuf_Module_GateProxy_query__E                         
8000c2a0  xdc_runtime_Main_Module_GateProxy_query__E                              
8000c2a0  xdc_runtime_System_Module_GateProxy_query__E                            
8000c2c0  ti_sysbios_gates_GateMutex_Instance_finalize__E                         
8000c2e0  ti_sysbios_BIOS_RtsGateProxy_query__E                                   
8000c2e0  ti_sysbios_gates_GateMutex_query__E                                     
8000c2e0  ti_sysbios_heaps_HeapMem_Module_GateProxy_query__E                      
8000c300  ti_sysbios_hal_Hwi_Module_startup__E                                    
8000c320  ti_sysbios_heaps_HeapMem_Module_GateProxy_enter__E                      
8000c340  ti_sysbios_heaps_HeapMem_Module_GateProxy_leave__E                      
8000c360  ti_sysbios_heaps_HeapMem_isBlocking__E                                  
8000c380  ti_sysbios_knl_Clock_TimerProxy_getMaxTicks__E                          
8000c3a0  ti_sysbios_knl_Idle_loop__E                                             
8000c3c0  ti_sysbios_knl_Queue_Instance_init__E                                   
8000c3e0  ti_sysbios_knl_Queue_Object__destruct__S                                
8000c400  ti_sysbios_knl_Queue_Object__get__S                                     
8000c420  ti_sysbios_knl_Queue_destruct                                           
8000c440  ti_sysbios_knl_Queue_empty__E                                           
8000c460  ti_sysbios_knl_Semaphore_Instance_finalize__E                           
8000c480  ti_sysbios_knl_Semaphore_destruct                                       
8000c4a0  ti_sysbios_knl_Swi_disable__E                                           
8000c4c0  ti_sysbios_knl_Task_disable__E                                          
8000c4e0  ti_sysbios_knl_Task_startup__E                                          
8000c500  ti_sysbios_knl_Clock_TimerProxy_Module__startupDone__S                  
8000c500  ti_sysbios_timers_dmtimer_Timer_Module__startupDone__F                  
8000c500  ti_sysbios_timers_dmtimer_Timer_Module__startupDone__S                  
8000c520  ti_sysbios_timers_dmtimer_Timer_getMaxTicks__E                          
8000c540  xdc_runtime_Error_getSite__E                                            
8000c560  xdc_runtime_Error_raiseX__E                                             
8000c580  xdc_runtime_Gate_enterSystem__E                                         
8000c5a0  xdc_runtime_Gate_leaveSystem__E                                         
8000c5c0  xdc_runtime_Memory_HeapProxy_alloc__E                                   
8000c5e0  xdc_runtime_Memory_HeapProxy_free__E                                    
8000c600  xdc_runtime_LoggerBuf_Module_GateProxy_enter__E                         
8000c620  xdc_runtime_LoggerBuf_Module_GateProxy_leave__E                         
8000c640  xdc_runtime_LoggerBuf_disable__E                                        
8000c660  xdc_runtime_LoggerBuf_enable__E                                         
8000c680  xdc_runtime_LoggerBuf_write1__E                                         
8000c6a0  xdc_runtime_LoggerBuf_write2__E                                         
8000c6c0  xdc_runtime_Memory_calloc__E                                            
8000c6e0  xdc_runtime_Memory_getMaxDefaultTypeAlign__E                            
8000c700  xdc_runtime_Startup_exec__I                                             
8000c720  xdc_runtime_Startup_rtsDone__E                                          
8000c740  xdc_runtime_SysMin_ready__E                                             
8000c740  xdc_runtime_System_SupportProxy_ready__E                                
8000c760  xdc_runtime_System_Module_GateProxy_enter__E                            
8000c780  xdc_runtime_System_Module_GateProxy_leave__E                            
8000c7a0  xdc_runtime_System_Module_startup__E                                    
8000c7c0  xdc_runtime_System_aprintf_va__E                                        
8000c7c0  xdc_runtime_System_aprintf_va__F                                        
8000c7e0  xdc_runtime_System_printf_va__E                                         
8000c7e0  xdc_runtime_System_printf_va__F                                         
8000c800  xdc_runtime_System_vsnprintf__E                                         
8000c820  xdc_runtime_Text_visitRope__I                                           
8000c840  xdc_runtime_Text_charTab__A                                             
8000ea00  ti_sysbios_family_c66_Cache_marvalues__C                                
8000ee00  xdc_runtime_Text_nodeTab__A                                             
8000f024  ti_sysbios_knl_Task_Object__PARAMS__C                                   
8000f060  xdc_runtime_LoggerBuf_Module__FXNS__C                                   
8000f09c  ti_sysbios_family_c62_TaskSupport_stackAlignment__C                     
8000f0a0  xdc_runtime_Startup_sfxnTab__A                                          
8000f100  ti_sysbios_heaps_HeapMem_Module__FXNS__C                                
8000f128  xdc_runtime_LoggerBuf_Object__PARAMS__C                                 
8000f150  ti_sysbios_gates_GateHwi_Module__FXNS__C                                
8000f174  ti_sysbios_gates_GateMutex_Module__FXNS__C                              
8000f198  ti_sysbios_heaps_HeapMem_Object__PARAMS__C                              
8000f1bc  ti_sysbios_knl_Semaphore_Object__PARAMS__C                              
8000f1e0  ti_sysbios_gates_GateHwi_Object__DESC__C                                
8000f200  ti_sysbios_gates_GateMutex_Object__DESC__C                              
8000f220  ti_sysbios_heaps_HeapMem_Object__DESC__C                                
8000f240  ti_sysbios_knl_Queue_Object__DESC__C                                    
8000f260  ti_sysbios_knl_Semaphore_Object__DESC__C                                
8000f280  ti_sysbios_knl_Task_Object__DESC__C                                     
8000f2a0  xdc_runtime_LoggerBuf_Object__DESC__C                                   
8000f2c0  xdc_runtime_Startup_sfxnRts__A                                          
8000f2da  ti_sysbios_family_c64p_Exception_Module__id__C                          
8000f2dc  ti_sysbios_gates_GateHwi_Object__PARAMS__C                              
8000f2f4  ti_sysbios_gates_GateMutex_Object__PARAMS__C                            
8000f30c  ti_sysbios_knl_Queue_Object__PARAMS__C                                  
8000f324  ti_sysbios_family_c64p_Exception_E_exceptionMax__C                      
8000f33a  ti_sysbios_family_c64p_Exception_useInternalBuffer__C                   
8000f344  ti_sysbios_knl_Idle_funcList__C                                         
8000f34c  ti_sysbios_family_c64p_Exception_exceptionHook__C                       
8000f350  xdc_runtime_Startup_firstFxns__A                                        
8000f358  xdc_runtime_Startup_firstFxns__C                                        
8000f360  xdc_runtime_Startup_lastFxns__C                                         
8000f368  ti_sysbios_family_c64p_Exception_externalHook__C                        
8000f36c  ti_sysbios_family_c64p_Exception_internalHook__C                        
8000f370  ti_sysbios_family_c64p_Exception_nmiHook__C                             
8000f374  ti_sysbios_family_c64p_Hwi_LD_end__C                                    
8000f378  ti_sysbios_family_c64p_Hwi_LM_begin__C                                  
8000f37c  ti_sysbios_family_c64p_Hwi_Module__diagsEnabled__C                      
8000f380  ti_sysbios_family_c64p_Hwi_Module__diagsIncluded__C                     
8000f384  ti_sysbios_family_c64p_Hwi_Module__diagsMask__C                         
8000f388  ti_sysbios_family_c64p_Hwi_Module__loggerFxn1__C                        
8000f38c  ti_sysbios_family_c64p_Hwi_Module__loggerFxn8__C                        
8000f390  ti_sysbios_family_c64p_Hwi_Module__loggerObj__C                         
8000f394  ti_sysbios_family_c66_Cache_E_invalidL1CacheSize__C                     
8000f398  ti_sysbios_family_c66_Cache_E_invalidL2CacheSize__C                     
8000f39c  ti_sysbios_family_c66_Cache_atomicBlockSize__C                          
8000f3a0  ti_sysbios_gates_GateMutex_A_badContext__C                              
8000f3a4  ti_sysbios_gates_GateMutex_Instance_State_sem__O                        
8000f3a8  ti_sysbios_gates_GateMutex_Module__diagsEnabled__C                      
8000f3ac  ti_sysbios_gates_GateMutex_Module__diagsIncluded__C                     
8000f3b0  ti_sysbios_gates_GateMutex_Module__diagsMask__C                         
8000f3b4  ti_sysbios_hal_Hwi_E_stackOverflow__C                                   
8000f3b8  ti_sysbios_heaps_HeapMem_A_align__C                                     
8000f3bc  ti_sysbios_heaps_HeapMem_A_heapSize__C                                  
8000f3c0  ti_sysbios_heaps_HeapMem_A_invalidFree__C                               
8000f3c4  ti_sysbios_heaps_HeapMem_A_zeroBlock__C                                 
8000f3c8  ti_sysbios_heaps_HeapMem_E_memory__C                                    
8000f3cc  ti_sysbios_heaps_HeapMem_Module__diagsEnabled__C                        
8000f3d0  ti_sysbios_heaps_HeapMem_Module__diagsIncluded__C                       
8000f3d4  ti_sysbios_heaps_HeapMem_Module__diagsMask__C                           
8000f3d8  ti_sysbios_heaps_HeapMem_Module__gateObj__C                             
8000f3dc  ti_sysbios_heaps_HeapMem_Object__count__C                               
8000f3e0  ti_sysbios_heaps_HeapMem_reqAlign__C                                    
8000f3e4  ti_sysbios_knl_Clock_LM_begin__C                                        
8000f3e8  ti_sysbios_knl_Clock_LM_tick__C                                         
8000f3ec  ti_sysbios_knl_Clock_LW_delayed__C                                      
8000f3f0  ti_sysbios_knl_Clock_Module_State_clockQ__O                             
8000f3f4  ti_sysbios_knl_Clock_Module__diagsEnabled__C                            
8000f3f8  ti_sysbios_knl_Clock_Module__diagsIncluded__C                           
8000f3fc  ti_sysbios_knl_Clock_Module__diagsMask__C                               
8000f400  ti_sysbios_knl_Clock_Module__loggerFxn1__C                              
8000f404  ti_sysbios_knl_Clock_Module__loggerFxn2__C                              
8000f408  ti_sysbios_knl_Clock_Module__loggerObj__C                               
8000f40c  ti_sysbios_knl_Semaphore_A_badContext__C                                
8000f410  ti_sysbios_knl_Idle_funcList__A                                         
8000f414  ti_sysbios_knl_Semaphore_A_noEvents__C                                  
8000f418  ti_sysbios_knl_Semaphore_A_overflow__C                                  
8000f41c  ti_sysbios_knl_Semaphore_A_pendTaskDisabled__C                          
8000f420  ti_sysbios_knl_Semaphore_Instance_State_pendQ__O                        
8000f424  ti_sysbios_knl_Semaphore_LM_pend__C                                     
8000f428  ti_sysbios_knl_Semaphore_LM_post__C                                     
8000f42c  ti_sysbios_knl_Semaphore_Module__diagsEnabled__C                        
8000f430  ti_sysbios_knl_Semaphore_Module__diagsIncluded__C                       
8000f434  ti_sysbios_knl_Semaphore_Module__diagsMask__C                           
8000f438  ti_sysbios_knl_Semaphore_Module__loggerFxn2__C                          
8000f43c  ti_sysbios_knl_Semaphore_Module__loggerFxn4__C                          
8000f440  ti_sysbios_knl_Semaphore_Module__loggerObj__C                           
8000f444  ti_sysbios_knl_Swi_LD_end__C                                            
8000f448  ti_sysbios_knl_Swi_LM_begin__C                                          
8000f44c  ti_sysbios_knl_Swi_LM_post__C                                           
8000f450  ti_sysbios_knl_Swi_Module__diagsEnabled__C                              
8000f454  ti_sysbios_knl_Swi_Module__diagsIncluded__C                             
8000f458  ti_sysbios_knl_Swi_Module__diagsMask__C                                 
8000f45c  ti_sysbios_knl_Swi_Module__loggerFxn1__C                                
8000f460  ti_sysbios_knl_Swi_Module__loggerFxn4__C                                
8000f464  ti_sysbios_knl_Swi_Module__loggerObj__C                                 
8000f468  ti_sysbios_knl_Swi_Object__count__C                                     
8000f46c  ti_sysbios_knl_Task_A_badPriority__C                                    
8000f470  ti_sysbios_knl_Task_A_badTaskState__C                                   
8000f474  ti_sysbios_knl_Task_A_badThreadType__C                                  
8000f478  ti_sysbios_knl_Task_A_badTimeout__C                                     
8000f47c  ti_sysbios_knl_Task_A_noPendElem__C                                     
8000f480  ti_sysbios_knl_Task_A_sleepTaskDisabled__C                              
8000f484  ti_sysbios_knl_Task_E_spOutOfBounds__C                                  
8000f488  ti_sysbios_knl_Task_E_stackOverflow__C                                  
8000f48c  ti_sysbios_knl_Task_LD_block__C                                         
8000f490  ti_sysbios_knl_Task_LD_exit__C                                          
8000f494  ti_sysbios_knl_Task_LD_ready__C                                         
8000f498  ti_sysbios_knl_Task_LM_sleep__C                                         
8000f49c  ti_sysbios_knl_Task_LM_switch__C                                        
8000f4a0  ti_sysbios_knl_Task_Module_State_inactiveQ__O                           
8000f4a4  ti_sysbios_knl_Task_Module__diagsEnabled__C                             
8000f4a8  ti_sysbios_knl_Task_Module__diagsIncluded__C                            
8000f4ac  ti_sysbios_knl_Task_Module__diagsMask__C                                
8000f4b0  ti_sysbios_knl_Task_Module__loggerFxn2__C                               
8000f4b4  ti_sysbios_knl_Task_Module__loggerFxn4__C                               
8000f4b8  ti_sysbios_knl_Task_Module__loggerObj__C                                
8000f4bc  ti_sysbios_knl_Task_Object__count__C                                    
8000f4c0  ti_sysbios_knl_Task_allBlockedFunc__C                                   
8000f4c4  ti_sysbios_knl_Task_defaultStackHeap__C                                 
8000f4c8  ti_sysbios_knl_Task_defaultStackSize__C                                 
8000f4cc  ti_sysbios_knl_Task_numConstructedTasks__C                              
8000f4d0  ti_sysbios_timers_dmtimer_Timer_E_cannotSupport__C                      
8000f4d4  ti_sysbios_timers_dmtimer_Timer_E_freqMismatch__C                       
8000f4d8  ti_sysbios_timers_dmtimer_Timer_Module__diagsEnabled__C                 
8000f4dc  ti_sysbios_timers_dmtimer_Timer_Module__diagsIncluded__C                
8000f4e0  ti_sysbios_timers_dmtimer_Timer_Module__diagsMask__C                    
8000f4e4  ti_sysbios_timers_dmtimer_Timer_numTimerDevices__C                      
8000f4e8  xdc_runtime_Assert_E_assertFailed__C                                    
8000f4ec  xdc_runtime_Core_A_initializedParams__C                                 
8000f4f0  xdc_runtime_Core_Module__diagsEnabled__C                                
8000f4f4  xdc_runtime_Core_Module__diagsIncluded__C                               
8000f4f8  xdc_runtime_Core_Module__diagsMask__C                                   
8000f4fc  xdc_runtime_Error_E_memory__C                                           
8000f500  xdc_runtime_Error_Module__diagsEnabled__C                               
8000f504  xdc_runtime_Error_Module__diagsIncluded__C                              
8000f508  xdc_runtime_Error_Module__diagsMask__C                                  
8000f50c  xdc_runtime_Error_Module__loggerFxn8__C                                 
8000f510  xdc_runtime_Error_Module__loggerObj__C                                  
8000f514  xdc_runtime_Error_policyFxn__C                                          
8000f518  xdc_runtime_Error_policy__C                                             
8000f51c  xdc_runtime_Error_raiseHook__C                                          
8000f520  xdc_runtime_IFilterLogger_Interface__BASE__C                            
8000f524  xdc_runtime_IGateProvider_Interface__BASE__C                            
8000f528  xdc_runtime_IHeap_Interface__BASE__C                                    
8000f52c  xdc_runtime_ILogger_Interface__BASE__C                                  
8000f530  xdc_runtime_IModule_Interface__BASE__C                                  
8000f534  xdc_runtime_Log_L_error__C                                              
8000f538  xdc_runtime_LoggerBuf_E_badLevel__C                                     
8000f53c  xdc_runtime_LoggerBuf_Module__gateObj__C                                
8000f540  xdc_runtime_LoggerBuf_Object__count__C                                  
8000f544  xdc_runtime_LoggerBuf_statusLogger__C                                   
8000f548  xdc_runtime_Memory_defaultHeapInstance__C                               
8000f54c  xdc_runtime_Startup_execImpl__C                                         
8000f550  xdc_runtime_Startup_maxPasses__C                                        
8000f554  xdc_runtime_Startup_sfxnRts__C                                          
8000f558  xdc_runtime_Startup_sfxnTab__C                                          
8000f55c  xdc_runtime_SysMin_bufSize__C                                           
8000f560  xdc_runtime_SysMin_outputFunc__C                                        
8000f564  xdc_runtime_System_Module__gateObj__C                                   
8000f568  xdc_runtime_System_abortFxn__C                                          
8000f56c  xdc_runtime_System_exitFxn__C                                           
8000f570  xdc_runtime_System_extendFxn__C                                         
8000f574  xdc_runtime_System_maxAtexitHandlers__C                                 
8000f578  xdc_runtime_Text_charTab__C                                             
8000f57c  xdc_runtime_Text_nameEmpty__C                                           
8000f580  xdc_runtime_Text_nameStatic__C                                          
8000f584  xdc_runtime_Text_nameUnknown__C                                         
8000f588  xdc_runtime_Text_nodeTab__C                                             
8000f58c  xdc_runtime_Text_visitRopeFxn__C                                        
8000f590  ti_sysbios_family_c64p_Hwi_Module__id__C                                
8000f592  ti_sysbios_family_c64p_Hwi_Module__loggerDefined__C                     
8000f594  ti_sysbios_family_c66_Cache_Module__id__C                               
8000f596  ti_sysbios_family_c66_Cache_registerRTSSynch__C                         
8000f598  ti_sysbios_gates_GateMutex_Module__id__C                                
8000f59a  ti_sysbios_hal_Hwi_Module__id__C                                        
8000f59c  ti_sysbios_heaps_HeapMem_Module__id__C                                  
8000f59e  ti_sysbios_knl_Clock_Module__id__C                                      
8000f5a0  ti_sysbios_knl_Clock_Module__loggerDefined__C                           
8000f5a2  ti_sysbios_knl_Semaphore_Module__id__C                                  
8000f5a4  ti_sysbios_knl_Semaphore_Module__loggerDefined__C                       
8000f5a6  ti_sysbios_knl_Swi_Module__id__C                                        
8000f5a8  ti_sysbios_knl_Swi_Module__loggerDefined__C                             
8000f5aa  ti_sysbios_knl_Task_Module__id__C                                       
8000f5ac  ti_sysbios_knl_Task_Module__loggerDefined__C                            
8000f5ae  ti_sysbios_timers_dmtimer_Timer_Module__id__C                           
8000f5b0  ti_sysbios_timers_dmtimer_Timer_checkFrequency__C                       
8000f5b2  ti_sysbios_timers_dmtimer_Timer_startupNeeded__C                        
8000f5b4  xdc_runtime_Core_Module__id__C                                          
8000f5b6  xdc_runtime_Error_Module__loggerDefined__C                              
8000f5b8  xdc_runtime_Error_maxDepth__C                                           
8000f5ba  xdc_runtime_LoggerBuf_Module__id__C                                     
8000f5bc  xdc_runtime_LoggerBuf_filterByLevel__C                                  
8000f5be  xdc_runtime_Memory_Module__id__C                                        
8000f5c0  xdc_runtime_SysMin_flushAtExit__C                                       
8000f5c2  xdc_runtime_Text_charCnt__C                                             
8000f5c4  xdc_runtime_Text_isLoaded__C                                            
8000f5c6  xdc_runtime_Text_registryModsLastId__C                                  
8000f5c8  xdc_runtime_Text_unnamedModsLastId__C                                   
8000f5d0  _stack                                                                  
800115d0  __TI_STACK_END                                                          
800115d0  ti_sysbios_heaps_HeapMem_Instance_State_0_buf__A                        
800125d0  ti_sysbios_knl_Task_Instance_State_0_stack__A                           
80012dd0  xdc_runtime_LoggerBuf_Instance_State_0_entryArr__A                      
80012fd0  xdc_runtime_SysMin_Module_State_0_outbuf__A                             
800131d8  ti_sysbios_BIOS_Module__state__V                                        
800131fc  ti_sysbios_family_c64p_Exception_Module__state__V                       
8001322c  ti_sysbios_family_c64p_Hwi_Module__root__V                              
80013234  ti_sysbios_family_c64p_Hwi_Module__state__V                             
800132a0  ti_sysbios_gates_GateHwi_Module__root__V                                
800132a8  ti_sysbios_gates_GateMutex_Module__root__V                              
800132b0  ti_sysbios_hal_Hwi_Module__root__V                                      
800132b8  ti_sysbios_heaps_HeapMem_Module__root__V                                
800132c0  ti_sysbios_knl_Clock_Module__root__V                                    
800132c8  ti_sysbios_knl_Clock_Module__state__V                                   
800132f4  ti_sysbios_knl_Queue_Module__root__V                                    
800132fc  ti_sysbios_knl_Semaphore_Module__root__V                                
80013304  ti_sysbios_knl_Swi_Module__root__V                                      
8001330c  ti_sysbios_knl_Swi_Module__state__V                                     
80013328  ti_sysbios_knl_Task_Module__root__V                                     
80013330  ti_sysbios_knl_Task_Module__state__V                                    
80013374  ti_sysbios_rts_ti_ThreadLocalStorage_Module__state__V                   
80013380  ti_sysbios_timers_dmtimer_Timer_Module__root__V                         
80013388  ti_sysbios_timers_dmtimer_Timer_Module__state__V                        
8001339c  xdc_runtime_Error_Module__state__V                                      
800133a0  xdc_runtime_LoggerBuf_Module__root__V                                   
800133a8  xdc_runtime_LoggerBuf_Module__state__V                                  
800133b0  xdc_runtime_Memory_Module__state__V                                     
800133b4  xdc_runtime_Registry_Module__state__V                                   
800133bc  xdc_runtime_Startup_Module__state__V                                    
800133c4  xdc_runtime_SysMin_Module__state__V                                     
800133d0  xdc_runtime_System_Module__state__V                                     
800133d8  xdc_runtime_Text_Module__state__V                                       
800133e0  __xdc__init__addr                                                       
800133e4  _lock                                                                   
800133e8  ti_sysbios_timers_dmtimer_Timer_Module_State_0_device__A                
800134a8  ti_sysbios_knl_Swi_Module_State_0_readyQ__A                             
80013528  ti_sysbios_knl_Task_Module_State_0_readyQ__A                            
800135a8  ti_sysbios_timers_dmtimer_Timer_Module_State_0_intFreqs__A              
80013628  ti_sysbios_timers_dmtimer_Timer_Object__table__V                        
80013688  ti_sysbios_knl_Task_Object__table__V                                    
800136d4  _unlock                                                                 
800136d8  ti_sysbios_gates_GateMutex_Object__table__V                             
80013718  ti_sysbios_timers_dmtimer_Timer_Module_State_0_handles__A               
80013758  ti_sysbios_knl_Swi_Object__table__V                                     
80013788  xdc_runtime_LoggerBuf_Object__table__V                                  
800137b0  ti_sysbios_family_c64p_Hwi_Object__table__V                             
800137c8  ti_sysbios_heaps_HeapMem_Object__table__V                               
800137e0  xdc_runtime_System_Module_State_0_atexitHandlers__A                     
800137f0  __TI_cleanup_ptr                                                        
800137f4  __TI_dtors_ptr                                                          
800137f8  __TI_enable_exit_profile_output                                         
80013800  ti_sysbios_hal_Hwi_Object__table__V                                     
80013808  ti_sysbios_gates_GateHwi_Object__table__V                               
80013810  ti_sysbios_knl_Task_Module_State_0_idleTask__A                          
80013818  __CIOBUF_                                                               
80013c00  ti_sysbios_family_c64p_Hwi0                                             
80013c00  ti_sysbios_family_c64p_Hwi_int0                                         
80013c20  ti_sysbios_family_c64p_Hwi_int1                                         
80013c40  ti_sysbios_family_c64p_Hwi_int2                                         
80013c60  ti_sysbios_family_c64p_Hwi_int3                                         
80013c80  ti_sysbios_family_c64p_Hwi_int4                                         
80013ca0  ti_sysbios_family_c64p_Hwi_int5                                         
80013cc0  ti_sysbios_family_c64p_Hwi_int6                                         
80013ce0  ti_sysbios_family_c64p_Hwi_int7                                         
80013d00  ti_sysbios_family_c64p_Hwi_int8                                         
80013d20  ti_sysbios_family_c64p_Hwi_int9                                         
80013d40  ti_sysbios_family_c64p_Hwi_int10                                        
80013d60  ti_sysbios_family_c64p_Hwi_int11                                        
80013d80  ti_sysbios_family_c64p_Hwi_int12                                        
80013da0  ti_sysbios_family_c64p_Hwi_int13                                        
80013dc0  ti_sysbios_family_c64p_Hwi_int14                                        
80013de0  ti_sysbios_family_c64p_Hwi_int15                                        
8001423c  __TI_Handler_Table_Base                                                 
80014248  __TI_Handler_Table_Limit                                                
80014250  __TI_CINIT_Base                                                         
80014260  __TI_CINIT_Limit                                                        
ffffffff  __TI_pprof_out_hndl                                                     
ffffffff  __TI_prof_data_size                                                     
ffffffff  __TI_prof_data_start                                                    
ffffffff  __binit__                                                               
ffffffff  __c_args__                                                              
ffffffff  binit                                                                   
UNDEFED   __TI_INITARRAY_Base                                                     
UNDEFED   __TI_INITARRAY_Limit                                                    
UNDEFED   __TI_TLS_INIT_Base                                                      
UNDEFED   __TI_TLS_INIT_Limit                                                     

[617 symbols]
